:104C29007584008539D2853AD3758401853BD2854F
:104C39003CD3E4F53AF5393000733056688566821D
:104C4900856583E0F56912822AE56C2539F539E530
:104C59006B353AF53AA3858266858365E5656563B3
:104C6900700AE56665647004D2668041E565641F73
:104C7900700CE56664FF700675660075650430584A
:104C89002C856482856383E56AF0A38582648583C4
:104C990063E563641F7016E56464FF701075640052
:104CA9007563048008853E3A853D39800030010CE2
:104CB900E539253FF539E53A3540F53A300206E55B
:104CC90033253AF53A300310E50A8536F0A425393B
:104CD900F539E5F0353AF53A300410E5118535F046
:104CE900A42539F539E5F0353AF53AE4F53CF53BD3
:104CF90030080D200908853E3C853D3B8002800037
:104D0900300A0CE53B253FF53BE53C3540F53C30A9
:104D19000B06E533253CF53C300C10E50A8536F0E9
:104D2900A4253BF53BE5F0353CF53C300D10E5118C
:104D39008535F0A4253BF53BE5F0353CF53C229063
:104D49004D8B302903124D58302A03124D6822E544
:0E4D59000B2509F50BE50C3508F50C93F50A52
:104D670022E512250EF512E513350DF51393C3133E
:104D7700F8E5142510F514E515350FF51593C3134C
:104D870028F511227F8285888C8F9295989B9EA10A
:104D9700A4A7AAADB0B3B6B9BBBEC1C3C6C9CBCE73
:104DA700D0D3D5D7D9DCDEE0E2E4E6E7E9EBEDEEF8
:104DB700F0F1F2F4F5F6F7F8F9FAFBFCFCFDFDFE6D
:104DC700FEFEFEFEFEFEFEFEFEFDFDFCFCFBFAFA0D
:104DD700F9F8F7F6F4F3F2F0EFEDECEAE8E7E5E3DC
:104DE700E1DFDDDBD8D6D4D1CFCDCAC8C5C2C0BDBF
:104DF700BAB7B4B2AFACA9A6A3A09D9A9794908D69
:104E07008A8784817E7A7774716E6B6865625F5C6E
:104E1700595653504D4A4744423F3C393734322F55
:104E27002D2A282624211F1D1B1918161412110FAD
:104E37000E0C0B0A08070605040403020201010011
:104E47000000000000000000000101020203040549
:104E5700060708090A0B0D0E1011131516181A1C50
:104E67001E20222427292B2E303335383A3D404245
:104E770045484B4E515456595C606366696C6F7276
:104E870075787B7FE537F5F0753D00E53EC39456B1
:104E97004013A4F5F0C394565007E5F02456F53EA9
:104EA70022753EAC227456953EA4F8C3945650061C
:104EB700745698F53E22753E0022E538F5F0B401A8
:104EC7000122753F00E540C394704020200907B4D4
:104ED700010475407022A420D20EF5F0C3947050DF
:104EE70007E5F02470F540227540FF22C3747095E2
:104EF70040200907B4010475407022A4F820D20BA2
:0F4F0700C394705006747098F5402275400022D4
:107C9B00D2F4C2F5C2F675840F85F0C81253F7748F
:107CAB0003127CEA1253E77403127CEA1253D612C6
:107CBB0053D67403127CEA1253D67402127CEA1266
:107CCB0053D67428127D597406127D59740E127D89
:107CDB00597401127D591253E77480127D5922C0D9
:107CEB0000A2E092F3A2E192F2A2E292F1A2E3925D
:107CFB00F0D2F475840F85F0C8C2F47830D8FE85C5
:107D0B00F0C87830D8FED00022C00075840FA2E4F2
:107D1B0092F3A2E592F2A2E692F1A2E792F0D2F4EC
:107D2B0085F0C8C2F47830D8FE85F0C87830D8FE1C
:107D3B00D00022203817EF75840FD2F5C2F685F0EC
:107D4B00C8127D141253D6127CEA1253D6227584B4
:107D5B000FC2F5C2F685F0C8127D141253D6127CF1
:107D6B00EA1253D62220380DEF14A2E492E6C2E4B5
:107D7B00D2E7127D5922740F127D5922740D127D98
:107D8B00592220380E7F01127D7078107F20127DD2
:107D9B003ED8F92220380E7F11127D7078107F208B
:067DAB00127D3ED8F92212
:10759F00C2B6758400D2C2C2C6D2C6C2C4D2C5C2D8
:1075AF00C330C3FD74A0F5C2C2C5C2C330C3FD8EC4
:1075BF00C2C2C330C3FD8FC2C2C330C3FD8DC2C2AE
:1075CF00C330C3FDD2C4C2C320C4FD1253E7D2B629
:1075DF0022758400C2C3D2C530C3FD74A0F5C2C2E8
:1075EF00C5C2C330C3FD8EC2C2C330C3FD8FC2C27A
:1075FF00C330C3FDC2C4D2C5C2C330C3FD74A1F52D
:10760F00C2C2C5C2C330C3FDC2C2C2C330C3FD852F
:10761F00C207D2C4C2C320C4FD22D2C2C2C6D2C6C0
:10762F00D2C4C2C320C4FD22758400D2C2C2C6D246
:10763F00C6C2C4D2C5C2C330C3FD74A0F5C2C2C591
:10764F00C2C330C3FD8EC2C2C330C3FD8FC2C2C31B
:10765F0030C3FD8C838D827B40E0A3F5C2C2C33063
:10766F00C3FDDBF5D2C4C2C320C4FD1253E722759C
:10767F008400C2C3D2C530C3FD74A0F5C2C2C5C257
:10768F00C330C3FD8EC2C2C330C3FD8FC2C2C3306D
:10769F00C3FDC2C4D2C5C2C330C3FD74A1F5C2C2FB
:1076AF00C5C2C330C3FD8C838D82C2C330C3FDE519
:1076BF00C2F0A31BBB01F3C2C2C2C330C3FDE5C2FC
:0976CF00F0D2C4C2C320C4FD22A4
:050003000248E232009A
:04000B00024C16325B
:10554A0075FF0775FFDE75FFAD75840F75E1077589
:10555A00E20475E34475840F75A43575A50975A62B
:10556A00BB75A7FF759CFF759D00759E00759FF022
:10557A0075D8FF75E8FF75F80F75AD0F758401755D
:10558A00893075888F75840275893075888F75841E
:10559A000F758A80758C67780874FF000000000018
:1055AA0000000000000000D5E0F1D8EDE58C30E7FE
:1055BA00FB759701758A0043890475840075B710D5
:1055CA0075840F438901758D01758F01758E02747B
:1055DA0080D5E0FD438902E58930E4FB75970275C1
:1055EA00840075D10775840075BB0175BA0075BC56
:1055FA00F075C70075C60075C5FF75C4FF75E881EB
:10560A0075840275BB0475BA0075BCF175C6007560
:10561A00C4FF75E88875840075D48475840175D4CF
:10562A0084758400C2F8759A47759D1A43F80975FE
:10563A00870075840075B90075A900759100759881
:10564A005075840175989075840075C04075C300C3
:10565A0075CFF2758400758E107589217588057568
:10566A008400758A00758BE0758CF4758DE043882B
:10567A004075840075C90075CA0075CB0075CC00E9
:10568A0075CD0075840175C91875CA8075CBFB750F
:10569A00CDFB75CC80D2CA75840275C91875CAA6A5
:1056AA0075CBAF75CDAF75CCA6D2CA75840075A877
:1056BA00AC75B81D75E6B075E71775F60075F74352
:1056CA0078A0760A76A1780A78A2760675A88590D7
:0656DA0000007F007E20AD
:1056E000E4F0A3DFFCDEFA7534327535FF7536C899
:1056F00078A0760A78A1760A78A27606D2B61276D3
:0257000029225C
:10536C0075840FD2FD2275840FC2FD2275840FD275
:10537C00FC2275840FC2FC2275840FD2FED234221B
:10538C0075840FC234C2FE22C29322D2932275843A
:10539C000FA2FA2275840FA2F92275840FA2DD22C6
:1053AC00A2922275840FA2DA2275840FA2DB2275D9
:1053BC00840FA2D82275840FA2D92200000000000D
:1053CC0000000000000000000022C000C0017904B1
:1053DC0078B4D8FED9FAD001D00022C000C0E07851
:1053EC009C7605E670FDD0E0D00022C000C0E078CD
:1053FC009C760FE670FDD0E0D00022C000C0E078B3
:10540C009C7664E670FDD0E0D00022EF75F06484E9
:10541C0024309000CBF0E5F0A375F00A842430F032
:10542C00A3E5F02430F022EF75F064842430900072
:10543C00CBF0E5F0A375F00A842430F0A3E5F0245A
:10544C0030F09000CBE0B4300B7420F0A3E0B4301B
:10545C00037420F022900021E0540FFFA3E0B4204D
:01546C00023D
:10546D008019540FCF75F00AA42FFFA3E0B42002CA
:10547D008009540FCF75F00AA42FFF22C006C00576
:10548D00C004900021E0540FFFFEA3E0B42003C33D
:10549D00802C540FFDCF75F00AA42FFFA3E0B4208C
:1054AD0003C3801A540FFCEE75F064A420D20EFED7
:1054BD00ED75F00AA42E40052C40028001D3D004D6
:1054CD00D005D0062275F06484F6E5F00875F00A73
:1054DD0084F608A6F008229000D1E075F009A42FFB
:1054ED00FFE5F03EFE79007A537B097C008E838FB9
:1054FD0082EC9389838A82F0A3A983AA820CDBEDC7
:10550D0022900057E0601775F010A42FF9EE35F0DA
:10551D00FA7BFFC006C00712ABFBD007D006900088
:10552D0058E0600F75F010A42FF9EE35F0FA7BFFFF
:0D553D0012A62122850607222285050622DE
:1000A600564F4950205441424C4520424547494EFF
:1000B60000564F4950205441424C452057524F4E0E
:1000C600470020564F4950205441424C4520454E4A
:1000D6004420002020202020202020202020202016
:1000E6002020205245504541544552204E554D4200
:1000F6004552202020202020202020203120746FEF
:10010600203230202053495445204E554D42455209
:100116002020202020202020202020203120746F25
:1001260020393982020011010215011482020111DF
:1001360003041501632020202020202020202020D9
:1001460020202020202020202020202020202020A9
:10015600202020202020434F5552544553592042F9
:100166004545502020204354435353204F4E2048AA
:10017600414E47202020205553455220454E4142AE
:100186004C452020202020524553455256452054A8
:100196004F4E45202020204E4554574F524B204D60
:1001A6004F44452020204E4554574F524B204E5524
:1001B6004D42455220202020202020202020202093
:1001C6002020202020202020202020202020202029
:1001D6002020202020202020202020202020202019
:1001E6002020202020202020202020202020202009
:1001F60020202020202020202020202020202020F9
:1002060020313D454E202020202020202020202067
:10021600204D4F4445202020202020202020202033
:1002260020544F4E4564010011020C150001640272
:100236000011030C15000164040011040C150001E3
:1002460064080011050C15000164100011060D1557
:100256000002C8030111070A1901012020202020ED
:100266002020202020202020202020202020202088
:10027600202020202020202020202020434F5552BF
:10028600544553592042454550202020435443535A
:1002960053204F4E2048414E47202020205553459D
:1002A6005220454E41424C452020202020524553A5
:1002B6004552564520544F4E45202020204E455449
:1002C600574F524B204D4F44452020204E45545702
:1002D6004F524B204E554D42455220202020202083
:1002E6002020202020202020202020202020202008
:1002F60020202020202020202020202020202020F8
:1003060020202020202020202020202020202020E7
:1003160020202020202020202020202020202020D7
:1003260020202020202020313D454E202020202046
:10033600202020202020204D4F4445202020202012
:1003460020202020202020544F4E45640100110219
:100356000C15000164020011030C15000164040071
:1003660011040C15000164080011050C1500016448
:10037600100011060D150001C8030111070A190125
:100386000120202020202020202020202020202086
:100396002020202020202020202020202020202057
:1003A6002020434F5552544553592042454550202D
:1003B6002020205553455220454E41424C45202091
:1003C600202043524F535320544F4E45204D4F4407
:1003D600452043544353532F4443532043524F53D2
:1003E6005320204E4554574F524B204D4F444520E5
:1003F60020204E4554574F524B204E554D424552A4
:1004060020202020202020202020202020202020E6
:1004160020202020202020202020202020313D4583
:100426004E2020202020202020202020204D4F4418
:1004360045202020202020202020202020544F4E00
:100446004520202020202020202020202020202081
:10045600206401001102091500016402001103095C
:1004660015000164040011060A150001C8030111F4
:10047600070C1901012020202020202020202020E8
:100486002020202020202020202020202020202066
:1004960020202020200101010101010101010000AD
:1004A6000000000000000000000000000000000046
:1004B6000000000000000000000000000000000036
:1004C6000000000000000000000000000000000026
:1004D6000000000000000000000000000000000016
:1004E60000000000000000000000000000000020E6
:1004F60020202020202020202020202020202020F6
:100506002020202020202020202020202020200104
:1005160001010101010101010000000000000000CD
:1005260000000000000000000000000000000000C5
:1005360000000000000000000000000000000000B5
:1005460000000000000000000000000000000000A5
:100556000000000000000000000000000000000095
:1005660000000000000000000020202020202020A5
:100576002020202020202020202020202020202075
:10058600202020202020202020010101010101013E
:100596000101202020202020202020202020202093
:1005A6002020202020202020202020202020202045
:1005B60020202054454C434F2050524F4752414D26
:1005C600202020524144494F2050524F4752414D1E
:1005D60020202050484F4E452050524F4752414D03
:1005E600202020434F4D50552050524F4752414DE9
:1005F6002020202041434345535320434F44452068
:10060600202044544D462054454C434F204C4556DB
:10061600454C44544D4620524144494F204C455682
:10062600454C4245455020524144494F204C455681
:10063600454C424545502054454C434F204C455669
:10064600454C4357494420524144494F204C455656
:10065600454C564F49434520524144494F204C454D
:10066600564C564F4943452054454C434F204C4524
:10067600564C5041474520524144494F204C45561F
:10068600454C435443535320524144494F204C4513
:10069600564C44435320524144494F204C455645FD
:1006A6004C204C545220524144494F204C4556450B
:1006B6004C2052505420524144494F204C455645F7
:1006C6004C2054454C434F20524144494F204C4501
:1006D600564C524144494F2054454C434F204C45BB
:1006E600564C524144494F204C494D4954204C45A3
:1006F600564C20434F53204F5220535155454C439F
:1007060048202020434F5320504F4C4152495459C2
:100716002020434F53205452494747455220564FB5
:100726004C54434F53204143515549535420544947
:100736004D45434F532052454C454153452054495E
:100746004D452053454E534520504F4C4152495438
:10075600592053454E205452494747455220564F3B
:100766004C5453454E204143515549535420544906
:100776004D4553454E2052454C454153452054491D
:100786004D45204C545220484F4C442044454C4142
:100796005920505454205455524E4F4646205449E1
:1007A6004D4552455045415445522054494D454FBB
:1007B60055542020414E54492D4B45524348554EE1
:1007C6004B202020535155454C4348205441494C19
:1007D60020202043544353532F44435320484F4C27
:1007E600442043524F535320425553592044454CBD
:1007F600415943524F5353204255535920484F4C69
:10080600442020204C54522053594E4320424954F0
:10081600202020414456414E43454420204C4F431E
:100826004B20202020202020202020202020202097
:1008360020202020202020202020202020202020B2
:1008460020202020202020202020202020202020A2
:100856002020202020202020202020202020202092
:100866002020202020202020202020202020313D54
:10087600454E202020202020202020202052415498
:10088600494F2020202020202020202020303D43BA
:100896004F532020202020202020202020313D5092
:1008A6004F532020202020202020202020203120CF
:1008B6004D532020202020202020202020313020B1
:1008C6004D53202020202020202020203130302091
:1008D6004D5320202020202020202020202020537F
:1008E600454320202020202020202020313D534B2E
:1008F6004950202020202020202020202020202099
:1009060020202020202020202020202020202020E1
:100916002020205052494F52495459204C455645A3
:100926004C20204C545220454E434F444520504FB6
:100936004C20204C5452204445434F444520504FB0
:100946004C2020205445535420494420434F4445CD
:10095600202049444C45204D45535341474520549A
:100966004D5220202020415245412042495420200A
:100976002020204D4153544552204F5220534C4184
:1009860056452044435320454E434F444520504F3F
:100996004C2020444353204445434F444520504F68
:1009A6004C2020434F5552544553592044454C4101
:1009B600592020202048414E472054494D452020AB
:1009C6002020434152524945522044524F50204420
:1009D6004C5920204143434553532044454C4159EB
:1009E600202053544154494F4E204944204D4F44F2
:1009F600452020564F494345204F522043574944EE
:100A060020202020494420494E54455256414C202E
:100A16002020202020435749442053504545442058
:100A260020202043574944204652455155454E43C0
:100A36005920202043574944204D455353414745AB
:100A46002020205455524E5F4F4E2044454C41596C
:100A56002020205455524E5F4F46462044454C4177
:100A660059202042454550204652455155454E4352
:100A7600592052455045415445522044495341421C
:100A86004C45204155582052454C4159204D4F4424
:100A960045202043524F53532042555359204D4F22
:100AA6004445205245504541544552204741494E00
:100AB6002020202054454C434F204741494E2020BA
:100AC60020204E4554574F524B2048414E475449DB
:100AD6004D45202020202020202020204C45564512
:100AE6004C2020202020202020202020303D4E4F4A
:100AF600524D202020202020202020202020434F3F
:100B06004445202020202020202020202020415243
:100B160045412020202020202020303D4D415354A7
:100B26004552202020202020202020202020312057
:100B36004D5320202020202020202020203130202E
:100B46004D5320202020202020202020313030200E
:100B56004D532020202020202020202031302053DB
:100B66004543202020202020202020202031204DF9
:100B7600494E2020202020202020202020204D4FBC
:100B86004445202020202020202020303D564F495B
:100B960043452020202020202020202020204652AF
:100BA6004551202020202020202020202020313DBB
:100BB600454E2020414C41524D20434F554E542026
:100BC600202020524553544F524520434F554E54F2
:100BD6002020202020494E54455256414C202020AA
:100BE6002020204E4554574F524B20434F4445201A
:100BF6002020494E544552434F4E4E454354204DB6
:100C06004F444E4554574F524B20494E4143544949
:100C1600564582010011022D1500018201011103C2
:100C26002D15000182010211042D15000182010318
:100C360011052D150001780604110601190101821E
:100C4600030A11072E1500FF82030B11082E15004B
:100C5600FF82030C11092E1500FF82030D110A2EC7
:100C66001500FF82030E110B2E1500FF82030F11D4
:100C76000C2E1500FF820310110D2E1500FF8203A6
:100C860011110E2E1500FF820312110F2E1500FFF3
:100C960082031311102E1500FF82031411112E1555
:100CA60000FF82031511122E1500FF820316111381
:100CB6002E1500FF82031711142E1500FF8203184C
:100CC60011152E1500FF82011911162F150001822C
:100CD600011A11173015000182031B11182E150079
:100CE600FF82021C11193115006382021D111A328E
:100CF60015006382011E111B3015000182031F11AE
:100D06001C2E1500FF820220111D31150063820280
:100D160021111E32150063820222111F3315026350
:100D26008203231120321501FF8203241121341579
:100D360002FF820225112233150063820226112347
:100D460032150063820227112433150363820228B9
:100D56001125321500638203291126331500FA8204
:100D6600012A11273515000182012B11385415016E
:100D76000982012C11395515000182012D113A55B0
:100D860015000182032E113B561501FA82032F111D
:100D96003C5C1500FF820130113D571500018201B0
:100DA60031113E58150001820132113F55160001DE
:100DB60082013311405515000182023411415A1542
:100DC600006382023511425B1500638202361143CD
:100DD6005A15006382023711445A1500638201389E
:100DE60011455E15000182013911465F1500018229
:100DF600023A11475D15006382023B1148591504FA
:100E06006382023C114960150114BE0A3D114A561F
:100E1600110000820247114B5A15006382024811E5
:100E26004D60150114820149114E5E1500028201C2
:100E36004A114F6115000182014B11505E150004E5
:100E460082014C11515415010982014D115254155C
:100E5600010982024E11533415006382014F11625B
:100E66000115000982015011630115000982025122
:100E760011645D150163C8035211650115010182F4
:100E8600015311665E150002820354116734150082
:100E9600FF01010200000200000200000000000045
:100EA6000101013132333435361432320532FFFF57
:100EB600FF1919196464C8FF000180000A01800047
:100EC6000A1E1AB400001E1E1E00010000020100C8
:100ED6000100000A1E630A000100050520202020EB
:100EE6002020202020200A05000000010114000017
:100EF600010000000044313233343536373839309A
:100F06002A2341424344AAA3C1C2C3C4D7ABA8A95A
:100F16002A23414243363330363730363934373177
:100F2600393734343737303739373832353835345E
:100F3600383835393135393438393734313030315C
:100F4600303331303731313031313431313831327B
:100F5600333132373133313133363134313134365E
:100F66003135313135363135393136323136353143
:100F76003637313731313733313737313739313821
:100F86003331383631383931393231393631393908
:100F96003230333230363231303231383232353225
:100FA600323932333332343132353032353430300F
:100FB6003630303730313530313730323130323308
:100FC60030323530323630333130333230333630FA
:100FD60034333034373035303035313035333035E1
:100FE60034303635303731303732303733303734C6
:100FF60031313431313531313631323231323531C8
:1010060033313133323133343134313134333134B5
:101016003531353231353531353631363231363591
:10102600313732313734323035323132323134328F
:101036003233323235323236323433323434323479
:101046003532343632353132353232353532363163
:10105600323633323635323636323731323734334A
:10106600303633313133313533323533333133334F
:10107600323334333334363335313335363336342D
:101086003336353337313431313431323431333428
:101096003233343331343332343435343436343510
:1010A60032343534343535343632343634343635F4
:1010B60034363635303335303635313635323335EC
:1010C60032363533323534363536353630363631D6
:1010D60032363234363237363331363332363534C9
:1010E60036363236363437303337313237323337B5
:1010F600333137333237333437343337353441428B
:10110600434445464748494A4B4C4D4E4F50515231
:10111600535455565758595A6162636465666768F1
:10112600696A6B6C6D6E6F707172737475767778B1
:10113600797A30313233343536373839607E21406A
:101146002324255E262A28295F2D2B3D7B7D5B5D8A
:101156007C3A3B3C3E2C2E3F2F2020202020202076
:10116600202020202020474C4F42414C2020202088
:1011760020202043544353533A202020202020206F
:101186002020204443533A202020202020202020C5
:1011960020202052455045415445522020202020F1
:1011A60020205350454544204449414C494E472050
:1011B600202053504545442043414C4C494E47203E
:1011C600202020505443204E554D42455220202089
:1011D600202020564F494345204D4553534147450E
:1011E600532020564F49434520504C4159424143D4
:1011F6004B202020494E56414C49442054595045D5
:10120600202020204F5554204F462052414E47451E
:10121600202020494C4C4547414C2056414C5545D1
:1012260020204D5553542046494C4C204649454CA8
:1012360044202020494C4C4547414C20434F4445CF
:1012460020202044415441204143434550544544C5
:1012560020204C494E45204E554D4245523A2020BD
:101266002020555345522050524F4752414D4D492B
:101276004E47204C54522049443A2020202020201A
:101286002020564F494345205245434F5244494E2C
:10129600472020494C4C4547414C20454E54525915
:1012A600202020494C4C4547414C2047414E472081
:1012B6002020202020434F4D504C455445442020AB
:1012C600202020474C4F42414C20454550524F4D1F
:1012D60020202020435443535320454550524F4D20
:1012E600202020202044435320454550524F4D2076
:1012F60020202020204C545220454550524F4D204E
:101306002020204449414C494E4720454550524FE4
:101316004D202043414C4C494E4720454550524FA5
:101326004D2020202050544320454550524F4D20FB
:1013360020202052455045415445522045455052A3
:101346004F4D2020494E495449414C495A494E4730
:101356002020202052455045415445523A20202015
:101366002020202020202020202020202020202077
:101376002020202020202020202020202020202067
:101386002020202020202020202020202020202057
:101396002020202020202020202020202020202047
:1013A600202020435443535320434F444520474174
:1013B6004E472044435320434F44452047414E4720
:1013C6002020205250545220434F44452047414E3E
:1013D600472020525054522047414E47202020207B
:0213E6002020C5
:107DB10030363230350912B23E12515102AAF81250
:107DC100B4BA128AC912A14012A19C12B3B43050A4
:107DD10005C250123D31129FC8E490022DF090026D
:107DE1002EF0C2362230372E30350512B26E803277
:107DF10012B4BA128AC912A14012A19C12B3B412D0
:107E01009FC8305005C250123D31E490022DF090D0
:107E1100022EF0C23722203803027EB53035061219
:107E21005BF602515130511A12B4BA128AC912A129
:107E31004012A19C12B3B4129FC8305005C2501217
:107E41003D31E490022DF090022EF0C2382059FD10
:107E5100900264747EF0D2592059FD9002647450EE
:107E6100F0D2592059FD9000D6E075F00A844430D3
:107E7100900264F0D2592059FD9000D6E075F00AC5
:107E810084E5F04430900264F0D2592059FD90020B
:107E910064305105745DF08003745BF0D259205950
:107EA100FD900264740DF0D2592059FD9002647462
:057EB1000AF0D2592285
:10515100900013E07012900014E0D394004009C253
:1051610036C237C238C23522900014E0127F8B520A
:105171008200528501528802528B03528E04529052
:1051810005529206529407529708529A0A529D0B61
:1051910052A00F52A31052A61152A91452AC15528B
:1051A100AF1652B21952B51A52B81B52BB1E52BE9B
:1051B1001F52C12352C42452C72852CA2952CD2D8D
:1051C10052D02E52D32F52D63052D93252DC3352D2
:1051D100DE3452E13552E43752E73852EA6452ED97
:1051E1006552F06652F36752F66E52F86F533A7099
:1051F10052FA7152FC7852FE79533A7A53007B533A
:105201000282530483533A8453068553098C530C09
:105211008D533A8E530E8F531196531497533A98D8
:105221005316995319A0531CA1533AA2531FA353C8
:1052310022AA5324AB533AAC5326AD5329B4532C71
:10524100B5533AB6532FB75331BE5334BF5337C05A
:10525100533AC1533CC2533FC85342C9533ACA534C
:1052610048CB534BF0534EF15351F25354FA535729
:10527100FB535AFC535DFD5360FE5363FF00005323
:105281006602B75202B5A202A36002B4E2800480B2
:1052910002800002A6F502625902AEF802B0410294
:1052A100AB38028B7402B07402AB77028A1C02B075
:1052B100A702ABB60285AB02B0DA02A40C02B10DB3
:1052C10002A46102B14002A4B602B17302B2FC02AF
:1052D100AE8602A73F12A2AE02A2548000029B44F6
:1052E10002A8E90299F302A0E402A02902A8A502FA
:1052F100AFA0025F2C8039804880408033801C80C1
:105301003A8005803C0266C8028736803402655FB8
:1053110002931D8006026DB802896C029AD5026063
:10532100C3800D801C0263ED028F28029D5D800BFE
:1053310002942F02A659028CC0800902825B028D61
:10534100F802972B02AD60029A6502B32A02840B20
:1053510002B775029CF302001202006A0200760293
:0B5361008E91020077E4900014F0220F
:10B75200E4900016F0900013741EF0900014E004C0
:02B76200F022D3
:10B5A200127D8D127D9F7BFF7A12796812ABFB7F31
:10B5B20011127D70C23CC239E4900016F090001462
:04B5C200E004F0228F
:10A36000303952900015E0FFC239BF2A079000141F
:10A37000E004F022BF5D0AC235E4900014F0D2512F
:10A3800022BF5B0AC235E4900014F0C25122BF2301
:10A39000247F23127D3E900016E004F0E0C3940475
:10A3A000400DC235E4900014F0127D8D027D9F9027
:05A3B00000147402F02E
:01A3B5002285
:10B4E2007BFF7A12796812ABFB127D9F7F11127D6E
:10B4F2007012002EE4900050F07F2A127D3EC23C72
:07B50200900014E004F022A8
:10A6F500303946900015E0F517C239E517642A6030
:10A7050038AF1712B7B55022AF17127D3E900050E3
:10A71500E02417F582E43400F583E517F090005046
:10A72500E004F0900014E004F0227BFF7A1279989F
:09A7350012ABFB90001474FAF061
:01A73E0022F8
:106259002039030263EC900015E0FFC239BF2A0719
:106269009000147403F022EF642360030263DD12CB
:106279007D3E900018E06439707CA3E06439707643
:10628900A3E064397070D23D900017E0FFB4310883
:10629900E490004AF002632FEFB43208E490004B17
:1062A900F0026347EFB433028043900017E0FFB474
:1062B9003408E490004CF0026375EFB43508E490BB
:1062C900004DF002638BEFB43608E490004EF00203
:1062D90063A1EFB437028015900017E0FFB43809C5
:1062E9009000497401F00263D6EFB4390B7BFF7A51
:1062F9001279A80263E3C23D900017E0FFB430169B
:10630900A3E0B43011A3E0B4300CA3E0B43007909B
:106319000014740AF022EFB43113900018E0B4307D
:106329000C12B5E95007900014740FF02290001771
:10633900E0B43211A3E0B4300C12B5E95007900073
:10634900147414F022900017E0B43311A3E0B430B0
:106359000C12B5E950079000147419F02290001737
:10636900E0B4340FA3E0B4300A12B6C49000147438
:106379001EF022900017E0B4350FA3E0B4300A12E2
:10638900B6D99000147423F022900017E0B4360FA8
:10639900A3E0B4300A12B6EE9000147428F02290EB
:1063A9000017E0B43716A3E0B43011A3E0B4300C01
:1063B900A3E0B43007900014742DF022900017E088
:1063C900B43811A3E0B4300C12B5E95007900014A9
:1063D9007437F0227BFF7A12799812ABFB90001484
:0363E90074FAF053
:0163EC00228E
:10AEF80090004F740BF09000507407F0E490005CE1
:10AF0800F0A3F090005E7402F0E490005FF0A3F00C
:10AF18007BFF7A11796812ABFB12A61B7F1E127D8C
:08AF2800709000147432F02255
:10B04100129894D39000D1E094019000D0E0940044
:10B05100400A12ABF590001474FAF0227E017F29A8
:10B061001254E47E007FD912550E900053E09000F7
:03B0710014F022B6
:10AB38007BFF7A11799812ABFB7BFF7A1179781237
:10AB4800A6217F0E127D70900019E0FF127D3E90C5
:10AB5800001AE0FF127D3E7F1A127D7090004F743C
:0FAB680010F09000507404F09000147432F0223A
:108B7400303E079000147403F02290001BE0643927
:108B84007041A3E06439703BA3E064397035900010
:108B94004F7411F09000507407F07BFF7A1379C87A
:108BA40012ABFBD23D900049E075F099A42469FE14
:108BB400E5F034FF90005CF0CE12A60C7F1E127D0F
:108BC40070804212A61B7F1E127D70129909503CC0
:108BD40090004F7411F09000507407F0900049E039
:108BE40075F099A42469FEE5F034FF90005CF0A3CD
:108BF400CEF090005E7403F090004AE0FF90005FB6
:108C0400E4F0A3EFF09000147432F02212ABF5906C
:068C1400001474FAF022C6
:10B07400129894D39000D1E094059000D0E094000D
:10B08400400A12ABF590001474FAF0227E027F2B72
:10B094001254E47E017F3B12550E900053E0900061
:03B0A40014F02283
:10AB77007BFF7A11799812ABFB7BFF7A11798812E8
:10AB8700A6217F0E127D70900019E0FF127D3E9086
:10AB9700001AE0FF127D3E7F1A127D7090004F74FD
:0FABA70015F09000507404F09000147432F022F6
:108A1C00303E079000147403F02290001BE0643980
:108A2C007042A3E06439703CA3E064397036900066
:108A3C004F7416F09000507407F07BFF7A1379C8CE
:108A4C0012ABFBD23D900049E0FF7E007C017D50D3
:108A5C00127F0EEF24A6FFEE340A12A6077F1E1219
:108A6C007D70804812A61B7F1E127D701297A45039
:108A7C004290004F7416F09000507407F09000492B
:108A8C00E0FF7E007C017D50127F0EEF24A6FFEEEE
:108A9C00340A90005CF0A3EFF090005E7403F09049
:108AAC00004BE0FF90005FE4F0A3EFF09000147433
:0D8ABC0032F02212ABF590001474FAF02293
:10B0A700129894D39000D1E094059000D0E09400DA
:10B0B700400A12ABF590001474FAF0227E037F5118
:10B0C7001254E47E027F6112550E900053E0900007
:03B0D70014F02250
:10ABB6007BFF7A11799812ABFB7BFF7A12797812B8
:10ABC600A6217F0E127D70900019E0FF127D3E9047
:10ABD600001AE0FF127D3E7F1A127D7090004F74BE
:0FABE6001AF09000507404F09000147432F022B2
:1085AB00303E079000147403F02290001BE06439F6
:1085BB007042A3E06439703CA3E0643970369000DC
:1085CB004F741BF09000507407F07BFF7A1379C83F
:1085DB0012ABFBD23D900049E0FF7E007C027DEEAA
:1085EB00127F0EEF2448FFEE342312A6077F1E12D4
:1085FB007D70806512A61B7F1E127D70129E979058
:10860B0000D2E0FEA3E0FFD39400EE94004051EFC4
:10861B0094FBEE9400504990004F741BF090005067
:10862B007407F0900049E0FF7E007C027DEE127F24
:10863B000EEF2448FFEE342390005CF0A3EFF09094
:10864B00005E7403F09000D3E024FFFE9000D2E0B4
:10865B0034FF90005FF0A3CEF09000147432F02240
:0A866B0012ABF590001474FAF0222F
:10B0DA00129894D39000D1E094039000D0E09400A9
:10B0EA00400A12ABF590001474FAF0227E047F57DE
:10B0FA001254E47E037F8712550E900053E09000AD
:03B10A0014F0221C
:10A40C0090004F741FF09000507407F090005C7433
:10A41C0060F0A374CEF0E490005EF090004CE0FF8E
:10A42C0090005FE4F0A3EFF07BFF7A1179A812ABF8
:10A43C00FB12A61B7F0F127D70900019E0FF127D9E
:10A44C003E90001AE0FF127D3E7F1E127D70900040
:05A45C00147432F0222F
:10B10D00129894D39000D1E094FF9000D0E094FF7A
:10B11D00400A12ABF590001474FAF0227E047F9B66
:10B12D001254E47E047F7B12550E900053E0900084
:03B13D0014F022E9
:10A4610090004F7424F09000507407F090005C74D9
:10A4710060F0A374CEF0E490005EF090004DE0FF38
:10A4810090005FE4F0A3EFF07BFF7A1179B812AB93
:10A49100FB12A61B7F0F127D70900019E0FF127D49
:10A4A1003E90001AE0FF127D3E7F1E127D709000EB
:05A4B100147432F022DA
:10B14000129894D39000D1E094FF9000D0E094FF47
:10B15000400A12ABF590001474FAF0227E057F15B8
:10B160001254E47E047FF512550E900053E09000D7
:03B1700014F022B6
:10A4B60090004F7429F09000507407F090005C747F
:10A4C60060F0A374CEF0E490005EF090004EE0FFE2
:10A4D60090005FE4F0A3EFF07BFF7A1179C812AB2E
:10A4E600FB12A61B7F0D127D70900019E0FF127DF6
:10A4F6003E90001AE0FF127D3E7F1E127D70900096
:05A50600147432F02284
:10B17300129894D39000D1E094FF9000D0E094FF14
:10B18300400A12ABF590001474FAF0227E057F8F0B
:10B193001254E47E057F6F12550E900053E0900029
:03B1A30014F02283
:10B2FC003038079000147401F02290004F742EF037
:10B30C009000507407F07BFF7A1179D812ABFB12C6
:0EB31C00A61B7F1E127D709000147432F0226A
:10AE8600303E07900014742FF02290001EE06438C4
:10AE96006005A3E0B4390A12ABF590001474FAF019
:10AEA600227BFF7A12798812ABFB90001EE0540FCA
:09AEB600F55A9000147430F022EA
:10A73F0090001EE064386005A3E0B4390A12ABF54F
:10A74F0090001474FAF0227BFF7A1179E812ABFBB8
:10A75F0090001EE0540FF55AD202D20B9000F8E091
:10A76F00F534125D927BFF7A1279B812ABFBC202FD
:09A77F00C20B90001474FEF022DC
:10A2AE0090001EE0540FF55A303602D200125DA413
:10A2BE0090026C7414F0C26730361B202704E542FE
:10A2CE0070F9125D9BC2007BFF7A1279B812ABFB5C
:10A2DE0090001474FEF030371F20250AE542600608
:10A2EE0012B72B3067F3125D9B7BFF7A1279B8128F
:08A2FE00ABFB90001474FEF0AC
:01A306002234
:10A25400303956900015E0FF900048F0C239127D65
:10A264003E900048E0FF12B7B55021900048E0FF4F
:10A27400900050E02417F582E43400F583EFF09069
:10A284000050E004F0900014E004F022900048E054
:10A29400B42A079000147403F0227BFF7A12799891
:0AA2A40012ABFB90001474FAF022D4
:109B440030396A900015E0FF900048F0C239127D68
:109B54003E900048E0FFB42A0B90004FE0900014C0
:109B6400F0D23E22EFB4230B90004FE0900014F0AB
:109B7400C23E22900048E0FF12B7B5502190004841
:109B8400E0FF900050E02417F582E43400F583EF01
:109B9400F0900050E004F0900014E004F0227BFF09
:0E9BA4007A12799812ABFB90001474FAF0223A
:10A8E90030393F900015E0FF900048F0127D3EC2DC
:10A8F90039900048E0FFB42A0B90004FE090001413
:10A90900F0D23E22EFB4230B90004FE0900014F0F8
:10A91900C23E227BFF7A12799812ABFB9000147425
:03A92900FAF0221F
:1099F30090004F7438F09000507407F090005C743E
:109A030060F0A374CEF090005E7456F0303D15E420
:109A130090005FF0A3F07BFF7A1379D812ABFB12AF
:109A2300A61B8032900049E024FFFEE434FF90003F
:109A33005FF0A3CEF07BFF7A13795812ABFB12A62B
:109A43001B7F0C127D70900019E0FF127D3E900089
:109A53001AE0FF127D3E7F1E127D70900014743257
:029A6300F022EF
:10A0E400129894D39000D1E094469000D0E094006C
:10A0F400400A12ABF590001474FAF0227E0C7F181B
:10A104001254E4900057E0FF601175F010A42498F5
:10A11400F9740535F0FA7BFF12ABFB900058E0FFB1
:10A12400601175F010A42498F9740535F0FA7BFFDA
:0CA1340012A621900053E0900014F022CD
:10A02900900056E0FF7003303E45127D7012B46611
:10A039001275E0900170EFF0900054E05F900170AC
:10A04900F060047F3180027F30127D3E303E20C2B5
:10A059003E900170E090003760057431F080037420
:10A0690030F09000477401F090001474F0F02290E1
:0EA079000059E0FF127D70900014E004F02208
:10A8A500303940900015E0FF900048F0C239127D24
:10A8B5003E900048E0FFB42A079000147403F0228C
:10A8C50012B7B5500F900048E0900021F0900014A9
:10A8D500E004F0227BFF7A12799812ABFB9000140A
:04A8E50074FAF022EF
:10AFA000303932900015E0FF900048F0C239BF2AD6
:10AFB000079000147403F022900048E0B423079037
:10AFC0000014E004F0227BFF7A12799812ABFB9018
:06AFD000001474FAF022E7
:105F2C00203D03025FBE900017E064386003025FFF
:105F3C00BE90005FF0A3F012B4669000D4EEF0A314
:105F4C00EFF01275E0900170EFF09000517401F0D9
:105F5C00900021E0B4311C900170E0FF900054E0FF
:105F6C00FEEF4E900170F0FD9000D4E0FEA3E0FF38
:105F7C0012759F900021E0B43018900054E0F4FFAB
:105F8C00900170E05FF0FD9000D4E0FEA3E0FF1202
:105F9C00759F900060E004F0700690005FE004F0E4
:105FAC00C3900060E0941490005FE094004088027D
:105FBC0060B3203D0302604F900017E06433600330
:105FCC0002604F90005FF0A3F012B4669000D4EE24
:105FDC00F0A3EFF01275E0900170EFF090005174A7
:105FEC0001F0900021E0B4311C900170E0FF9000B2
:105FFC0054E0FEEF4E900170F0FD9000D4E0FEA353
:10600C00E0FF12759F900021E0B43018900054E02E
:10601C00F4FF900170E05FF0FD9000D4E0FEA3E08F
:10602C00FF12759F900060E004F0700690005FE036
:10603C0004F0C3900060E094FA90005FE09400409C
:10604C0088805D12B4669000D4EEF0A3EFF0127568
:10605C00E0900170EFF09000517401F0900021E09D
:10606C00B4311E900170E0FF900054E0FEEF4E90B2
:10607C000170F0FD9000D4E0FEA3E0FF12759F804C
:10608C001F900021E0B4301F900054E0F4FF900109
:10609C0070E05FF0FD9000D4E0FEA3E0FF12759F6E
:1060AC0090001474FEF0227BFF7A12799812ABFBED
:0760BC0090001474FAF022B9
:10942F00900056E0FF7003303E68127D7012B466F4
:10943F009000D4EEF0A3EFF0E4900170F0900054A0
:10944F00E0FF900170E0C39F50349000D4E475F0BA
:10945F0001127F75AFF0FE1275E0900171E4F0A379
:10946F00EFF0E0FF900170E02437F582E43400F56F
:10947F0083EFF0127D3E900170E004F080BF303E2C
:10948F0011C23E900054E0900047F090001474F029
:10949F00F022900050740AF0900059E0FF127D7096
:0794AF00900014E004F0221C
:10972B00303975900015E0FF900048F0C239127D7A
:10973B003E900048E0FFB42A079000147403F02217
:10974B00EFB42308900014E004F0803912B7B55041
:10975B0038900048E0FF900050E0FE04F074172EA4
:10976B00F582E43400F583EFF0900054E02409FF18
:10977B00E433FE900050E0D39FEE6480F874809841
:10978B004016900014E004F0227BFF7A12799812B5
:09979B00ABFB90001474FAF022FB
:10AD6000303937900015E0FF900048F0C239127D6D
:10AD70003E900048E0FFB42A079000147403F022CC
:10AD8000EFB42307900014E004F0227BFF7A1279DD
:0BAD90009812ABFB90001474FAF02244
:10825B00303D7B900017E06433707390005FF0A3A8
:10826B00F012B4669000D4EEF0A3EFF090005074CF
:10827B000AF0E4900170F0900054E0FF900170E080
:10828B00C39F502B9000D4E475F001127F75AFF0B3
:10829B00FE900050E0FD04F074172DF582E43400DD
:1082AB00F583E0FD12759F900170E004F080C8909B
:1082BB000060E004F0700690005FE004F0C39000F3
:1082CB0060E094FA90005FE094004095804E12B409
:1082DB00669000D4EEF0A3EFF0900050740AF0E437
:1082EB00900170F0900054E0FF900170E0C39F503C
:1082FB002B9000D4E475F001127F75AFF0FE900067
:10830B0050E0FD04F074172DF582E43400F583E0A2
:10831B00FD12759F900170E004F080C87BFF7A120C
:0C832B0079B812ABFB90001474FEF02235
:109AD50030396B900015E0FF900048F0C239127DD7
:109AE5003E900048E0FFB42A079000147403F0226A
:109AF50012B7B5501A900048E0FF900050E0FE0400
:109B0500F074172EF582E43400F583EFF080107BB6
:109B1500FF7A12799812ABFB90001474FAF0229038
:109B25000054E02409FFE433FE900050E0D39FEE9B
:0F9B35006480F87480984006900014E004F022D9
:10873600900056E0FF7006203E030287E1127D702E
:1087460012B4669000D4EEF0A3EFF01275E0125466
:1087560033900054E0B401109000CDE0FF127D3E4E
:108766009000CDE0900037F0900054E0B4022090E5
:1087760000CCE0FF127D3E9000CDE0FF127D3E90E2
:1087860000CCE0900037F09000CDE0900038F090FB
:108796000054E0640370309000CBE0FF127D3E9001
:1087A60000CCE0FF127D3E9000CDE0FF127D3E90B2
:1087B60000CBE0900037F09000CCE0900038F090CD
:1087C60000CDE0900039F0303E11C23E900054E0FA
:1087D600900047F090001474F0F022900059E0FFEA
:1087E600127D70900050740AF0900014E004F0229C
:1066C8001254895003026824125461900170EFF04B
:1066D80090005AE0FEEFC39E5003026824A3E0FF37
:1066E800900170E0D39F4003026824303D41900040
:1066F80017E06431703990005FF0A3F012B466902F
:1067080000D4EEF0A3EFF0900170E0FD12759F90B9
:106718000060E004F0700690005FE004F0C39000B1
:1067280060E0943390005FE0940040D00268143039
:106738003D41900017E06432703990005FF0A3F09B
:1067480012B4669000D4EEF0A3EFF0900170E0FD73
:1067580012759F900060E004F0700690005FE004FE
:10676800F0C3900060E0947090005FE0940040D027
:10677800026814303D40900017E064337038900090
:106788005FF0A3F012B4669000D4EEF0A3EFF0909F
:106798000170E0FD12759F900060E004F0700690B3
:1067A800005FE004F0C3900060E094FA90005FE0BE
:1067B800940040D08056303D40900017E064387017
:1067C8003890005FF0A3F012B4669000D4EEF0A306
:1067D800EFF0900170E0FD12759F900060E004F00A
:1067E800700690005FE004F0C3900060E09414909D
:1067F800005FE0940040D0801312B4669000D4EE9D
:10680800F0A3EFF0900170E0FD12759F7BFF7A1204
:1068180079B812ABFB90001474FEF02212ABF5901D
:06682800001474FAF022D6
:10655F0012548950030266BE125461900170EFF01D
:10656F0090005AE0FEEFC39E400BA3E0FF90017036
:10657F00E0D39F4009900170E060030266BE303D9A
:10658F0041900017E06431703990005FF0A3F01272
:10659F00B4669000D4EEF0A3EFF0900170E0FD121E
:1065AF00759F900060E004F0700690005FE004F0CB
:1065BF00C3900060E0943390005FE0940040D002FD
:1065CF0066AE303D41900017E06432703990005F45
:1065DF00F0A3F012B4669000D4EEF0A3EFF09001A8
:1065EF0070E0FD12759F900060E004F0700690005F
:1065FF005FE004F0C3900060E0947090005FE0945F
:10660F000040D00266AE303D40900017E06433701A
:10661F003890005FF0A3F012B4669000D4EEF0A3B0
:10662F00EFF0900170E0FD12759F900060E004F0B4
:10663F00700690005FE004F0C3900060E094FA9061
:10664F00005FE0940040D08056303D40900017E04E
:10665F006438703890005FF0A3F012B4669000D4E5
:10666F00EEF0A3EFF0900170E0FD12759F900060C7
:10667F00E004F0700690005FE004F0C3900060E06B
:10668F00941490005FE0940040D0801312B4669091
:10669F0000D4EEF0A3EFF0900170E0FD12759F7B38
:1066AF00FF7A1279B812ABFB90001474FEF022122D
:0966BF00ABF590001474FAF0220E
:10931D00900056E0FF7003303E6A127D7012B46605
:10932D009000D4EEF0A3EFF01275E0900170EFF025
:10933D001294B6E4900170F0900170E0FFC39404B4
:10934D005030E0FE24CBF582E43400F583E0FD746B
:10935D00372EF582E43400F583EDF074CB2FF582D2
:10936D00E43400F583E0FF127D3E900170E004F0DF
:10937D0080C6303E0FC23E9000477403F09000143B
:10938D0074F0F022900059E0FF127D70900050743F
:09939D000AF0900014E004F02233
:106DB8007F0A127A54900170EFF07003026EEF3080
:106DC8003D42900017E06431703A90005FF0A3F004
:106DD80012B4669000D4EEF0A3EFF0900170E014C6
:106DE800FD12759F900060E004F0700690005FE06F
:106DF80004F0C3900060E0943390005FE09400409A
:106E0800CF026ED7303D42900017E06432703A905E
:106E1800005FF0A3F012B4669000D4EEF0A3EFF098
:106E2800900170E014FD12759F900060E004F0700E
:106E38000690005FE004F0C3900060E0947090005A
:106E48005FE0940040CF026ED7303D41900017E0DC
:106E58006433703990005FF0A3F012B4669000D4E8
:106E6800EEF0A3EFF0900170E014FD12759F900012
:106E780060E004F0700690005FE004F0C3900060EA
:106E8800E094FA90005FE0940040CF8042303D43A8
:106E9800900017E06438703B90005FF0A3F012B4E4
:106EA800669000D4EEF0A3EFF0900170E014FD12AC
:106EB800759F900060E004F0700690005FE004F0B9
:106EC800C3900060E0941490005FE0940040CF7B92
:106ED800FF801C12B4669000D4EEF0A3EFF090018E
:106EE80070E014FD12759F900170E07BFF600E7AD0
:106EF8001279B812ABFB90001474FEF0227A127962
:0B6F08003812ABFB90001474FAF0226A
:10896C00900056E0FF7006203E03028A07127D70CD
:10897C0012B4669000D4EEF0A3EFF01275E012542E
:10898C00339000D4E475F001127F75AFF0FE1275D0
:10899C00E01254179000CCE0FF900037F0A3F012D7
:1089AC007D3E9000CDE0FF127D3E9000D4E475F04A
:1089BC0001127F75AFF0FE1275E01254179000CBC8
:1089CC00E0FF900039F09000CCE090003AF090007D
:1089DC00CDE090003BF0127D3E9000CCE0FF127D8C
:1089EC003E9000CDE0FF127D3E303E0FC23E900027
:1089FC00477405F090001474F0F022900059E0FFD9
:108A0C00127D70900050740AF0900014E004F02273
:1060C300900021E0540F75F00AA4FFA3E0540F2FB2
:1060D300900170F0FD900024E0540F75F00AA4FBCA
:1060E300AAF0900023E0540F75F064A42BFFE5F0B1
:1060F3003AFE900025E0540F7A002FFFEA3E90010C
:1061030074F0A3EFF0EDC394014022900170E0D34B
:1061130094145019900174E0FEA3E0FFC39401EEC0
:1061230094004009D3EF94FAEE9400400A12ABF5C1
:1061330090001474FAF022303D5E900017E0643151
:10614300705690005FF0A3F012B4669000D4EEF0A6
:10615300A3EFF09000D4E475F001127F75AFF0FE69
:10616300900170E0FD12759F9000D4E0FEA3E0FF64
:10617300900175E0FD12759F900060E004F07006D9
:1061830090005FE004F0C3900060E0943390005F00
:10619300E0940040B3026249303D5D900017E06433
:1061A30032705590005FF0A3F012B4669000D4EE05
:1061B300F0A3EFF09000D4E475F001127F75AFF017
:1061C300FE900170E0FD12759F9000D4E0FEA3E005
:1061D300FF900175E0FD12759F900060E004F07080
:1061E3000690005FE004F0C3900060E094709000BC
:1061F3005FE0940040B3804E12B4669000D4EEF09A
:10620300A3EFF09000D4E475F001127F75AFF0FEB8
:10621300900170E0FD12759F900024E0540F75F01B
:106223000AA4FF900023E0540F75F064A42FFF909D
:106233000025E0540F2F900170F0FD9000D4E0FE94
:10624300A3E0FF12759F7BFF7A1279B812ABFB9024
:06625300001474FEF022AD
:1063ED007F0D127A54EF701A900024E0B43010A390
:1063FD00E0B4300BA3E0B43006A3E06430600302D8
:10640D0064F7900028E0FF64306004EFB4350E901F
:10641D000029E0540FD3940540030264F79000283F
:10642D00E0FF64316004EFB4361190002DE0B4202C
:10643D000790002CE0B420030264F7900028E0FFE1
:10644D0064326004EFB4371190002CE0B420079053
:10645D00002BE0B420030264F7900028E0FF6433C2
:10646D006004EFB43809900029E0B42002807B90DD
:10647D000028E0FF64346005EF64397077900029DF
:10648D00E0540F75F00AA4FFA3E0540F2F90017094
:10649D00F0FD90002CE0540F75F00AA4FBAAF090CB
:1064AD00002BE0540F75F064A42BFFE5F03AFE903D
:1064BD00002DE0540F7A002FFFEA3E900174F0A3F7
:1064CD00EFF0EDC394014022900170E0D39414508D
:1064DD0019900174E0FEA3E0FFC39401EE94004017
:1064ED0009D3EF94FAEE9400400A12ABF590001424
:1064FD0074FAF02212B4669000D4EEF0A3EFF0908F
:10650D000050740AF0E4900170F0900054E0FF9098
:10651D000170E0C39F502B9000D4E475F001127F01
:10652D0075AFF0FE900050E0FD04F074172DF5826C
:10653D00E43400F583E0FD12759F900170E004F0E6
:10654D0080C87BFF7A1279B812ABFB90001474FEF1
:02655D00F0222A
:108F2800900056E0FF7003303E73127D7012B466F5
:108F38009000D4EEF0A3EFF0E4900170F0900054AC
:108F4800E0FF900170E0C39F503F9000D4E475F0BB
:108F580001127F75AFF0FE1275E0900171E4F0A385
:108F6800EFF0E0FF900170E02437F582E43400F57B
:108F780083EFF0900171E0FEA3E0FF1275E0127D2F
:108F88003E900170E004F080B4303E11C23E900083
:108F980054E0900047F090001474F0F022900059CB
:108FA800E0FF127D70900050740AF0D23C900014DB
:048FB800E004F022BF
:109D5D00303965900015E0FF900048F0C239BF2AF8
:109D6D00079000147403F022900048E0FFB423081C
:109D7D00900014E004F0803DEF547FFF127D3E9083
:109D8D000048E0547FFF900050E0FE04F074172E61
:109D9D00F582E43400F583EFF0900054E02409FFE0
:109DAD00E433FE900050E0D39FEE6480F874809809
:099DBD004006900014E004F022BD
:10A6590030394B900015E0FF900048F0C239BF2A0D
:10A66900079000147403F022900048E0FFB4230B14
:10A67900900014E004F0E004F0801012B7B5500F18
:10A68900900048E0900052F0900014E004F0227B22
:0FA69900FF7A12799812ABFB90001474FAF0223A
:108CC000203903028D5C900015E0FF900048F0C24F
:108CD00039BF2A079000147403F022900048E0FF87
:108CE000B4230A900014E004F0E004F02212B7B5B7
:108CF000505B900052E0540F75F00AA4FF900048BA
:108D0000E0540F2FF0E090110493FF900048F01210
:108D10007D3E900048E0FF900050E0FE04F07417A4
:108D20002EF582E43400F583EFF0900054E024093E
:108D3000FFE433FE900050E0D39FEE6480F874802F
:108D400098900014E0400304F02214F0227BFF7A94
:0D8D500012799812ABFB90001474FAF02217
:108DF800900056E0FF7003303E7A127D7012B46620
:108E08009000D4EEF0A3EFF01275E0C0079000D503
:108E1800E02401FF9000D4E03400FE1275E0AD07B5
:108E2800D007125546900061EEF0A3EFF012A6A805
:108E38009000CBE0FF127D3E9000CCE0FF127D3E1B
:108E48009000CDE0FF127D3E9000CBE0900037F01F
:108E58009000CCE0900038F09000CDE0900039F020
:108E6800303E11C23E900054E0900047F09000144C
:108E780074F0F022900059E0FF127D709000507459
:098E88000AF0900014E004F0224D
:109A650012B20C900171EEF0A3EFF0D394E7EE94EF
:109A7500035053D25012B4669000D4EEF0A3EFF029
:109A8500900171E0FEA3E0FF125545AD079000D4AB
:109A9500E0FEA3E0FF12759F900171E0FEA3E0FFD9
:109AA500125541AD079000D5E02401FF9000D4E0A8
:109AB5003400FE12759F7BFF7A1279B812ABFB90CA
:109AC500001474FEF02212ABF590001474FAF02223
:10B32A0030360B900120E0900006F012536C303852
:10B33A0005E4900006F030370E90000630340574AC
:0EB34A000AF080037428F0900014E004F02252
:10840B00900006E060030284DC12780630383E20D0
:10841B0059FD900264747EF0D2592059FD9002648C
:10842B007450F0D2592059FD9000D6E075F00A84B3
:10843B004430900264F0D2592059FD9000D6E0757B
:10844B00F00A84E5F04430900264F0D25990005366
:10845B00E0127F8B84846484896E8489788489821A
:10846B0084898C848B968490A08495AA849AB484F6
:10847B009FBE8489C8000084A712B509801E80198D
:10848B0012AC70801712ACAC8012120078800D12F7
:10849B000079800812AA78800312A5B430360F90A9
:1084AB00010CE0900001F0900014E004F022303851
:1084BB001A2059FD900264740DF0D2592059FD9089
:1084CB000264740AF0D259C238C235900014740198
:0284DB00F0228D
:10B77500900001E070091253729000147401F022D8
:109CF300303611900120E0900006F012536C900072
:109D030006E070FA30370C9000067405F0900006F8
:109D1300E070FAE4900170F030370C12B83012544E
:109D23000712B85A12540730360C12B83B125407B4
:109D330012B85A125407900170E004F0E0C394057E
:109D430040D630360E90010CE0900001F0900001F7
:0A9D5300E070FA9000147401F02291
:0100120022CB
:01006A002273
:010076002267
:108E91003038079000147402F02230370A2034076A
:108EA1009000147401F022303611900120E09000FE
:108EB10006F012536C900006E070FA30370C900007
:108EC100067405F0900006E070FA3036209000F547
:108ED100E0F53612B83BE4900170F01254079001AE
:108EE10070E004F0E0C3940A40F112B85A30372020
:108EF1009000F6E0F53612B830E4900170F01254AB
:108F010007900170E004F0E0C3940A40F112B85AEE
:108F110030360E90010CE0900001F0900001E070FD
:078F2100FAE4900014F022B5
:010077002266
:10B23E0030272C203929900013741EF0787EE6FFFB
:10B24E00547FFE900EFB93900015F0303C0DEF30C6
:10B25E00E709EE900F0B93900015F0D239C227221A
:10B26E0030252C203929900013741EF0787CE6FFCF
:10B27E00547FFE900EFB93900015F0303C0DEF3096
:10B28E00E709EE900F0B93900015F0D239C22522EC
:105BF600900274E0FF65797003025D91303903020B
:105C06005D91900013741EF0EFD394FA4005E49072
:105C16000274F0900274E0FF04F074752FF582E4CC
:105C26003402F583E0FF647F7003025D91D239BFD1
:105C36005D07900015745DF022BF5B079000157438
:105C46005BF022BF30079000157430F022BF310799
:105C56009000157431F022BF32079000157432F0AF
:105C660022BF33079000157433F022BF340790002B
:105C7600157434F022BF35079000157435F022BF35
:105C860036079000157436F022BF3707900015745A
:105C960037F022BF38079000157438F022BF390755
:105CA6009000157439F022BF23079000157423F075
:105CB60022BF2A07900015742AF022BF41079000E0
:105CC600157441F022BF42079000157442F022BFBE
:105CD60043079000157443F022BF640790001574C3
:105CE60044F022203C03C23922BF6107900015749C
:105CF60061F022BF62079000157462F022BF63074D
:105D06009000157463F022BF64079000157464F068
:105D160022BF65079000157465F022BF66079000E4
:105D2600157466F022BF67079000157467F022BFEE
:105D360068079000157468F022BF69079000157413
:105D460069F022BF6A07900015746AF022BF6B07DC
:105D5600900015746BF022BF6C07900015746CF000
:105D660022BF6D07900015746DF022BF6E0790007C
:105D760015746EF022BF6F07900015746FF022BF86
:0B5D860070079000157470F022C23905
:015D910022EF
:10002E00E4900170F0900170E0FFC39420501574BD
:10003E00172FF582E43400F5837420F0900170E000
:05004E0004F080E12236
:0FB7B500EFC394304007EFD39439500122C322E1
:10989400900020E0FD6420602E90001FE0540F75BE
:1098A400F00AA4FBAAF090001EE0540F75F064A423
:1098B4002BFFE5F03AFEED540F7C002FFFEC3E90B9
:1098C40000D0F0A3EF803190001FE0FD64209000F1
:1098D4001E601AE0540F75F00AA4FFED540F7C00CB
:1098E4002FFEEC35F09000D0F0A3CE800BE0540FA7
:1098F400FF9000D0E4F0A3EFF0E024FFF09000D05C
:05990400E034FFF02239
:109E970090001DE0FD6420602B90001CE0540F75BE
:109EA700F00AA4FBAAF090001BE0540F75F064A41D
:109EB7002BFFE5F03AFEED540F7C002FFFEC3E90B0
:109EC70000D2802E90001CE0FD642090001B601AD9
:109ED700E0540F75F00AA4FFED540F7C002FFEEC41
:109EE70035F09000D2F0A3CEF022E0540FFF90009F
:079EF700D2E4F0A3EFF0221A
:10B5E900900019E0540F75F00AA4FFA3E0540F2F3F
:10B5F900900049F0D394004006E09415500122C30D
:01B60900221E
:10990900E4900170F0900170E0FFC394335064EF6C
:1099190075F003A4241BF582E4340FF583E493FF67
:1099290090001BE0FEEF6E7042900170E0FF75F051
:1099390003A4241CF582E4340FF583E493FE90001C
:109949001CE0FDEEB50524EF75F003A4241DF58296
:10995900E4340FF583E493FF90001DE0FEEFB506B4
:109969000A900170E090004AF0D322900170E0045F
:05997900F08092C32202
:1097A400E4900170F0900170E0FFC394705067750D
:1097B400F003EFA424B4F582E5F0340FF583E493C9
:1097C400FF90001BE0FEEF6E7044900170E0FF75A7
:1097D400F003A424B5F582E5F0340FF583E493FE99
:1097E40090001CE0FDEEB5052575F003EFA424B64A
:1097F400F582E5F0340FF583E493FF90001DE0FE5D
:10980400EFB5060A900170E090004BF0D32290016E
:0898140070E004F0808FC32214
:107A540074172FF582E43400F583E0FE643160038B
:107A6400027AE8900170F0900170E0FDC394335005
:107A74007074182FF582E43400F583E0FCED75F0A2
:107A840003A4241BF582E4340FF583E4936C70495A
:107A940074192FF582E43400F583E0FD900170E061
:107AA400FC75F003A4241CF582E4340FF583E493FD
:107AB400B50526741A2FF582E43400F583E0FDEC55
:107AC40075F003A4241DF582E4340FF583E493B523
:107AD4000507900170E004FF22900170E004F0803B
:107AE400867F0022EE64326003027B75900170F0A1
:107AF400900170E0FEC39470507474182FF582E402
:107B04003400F583E0FD75F003EEA424B4F582E5BA
:107B1400F0340FF583E4936D704C74192FF582E4FF
:107B24003400F583E0FE900170E0FD75F003A424B9
:107B3400B5F582E5F0340FF583E493B50628741A9D
:107B44002FF582E43400F583E0FE75F003EDA42400
:107B5400B6F582E5F0340FF583E493B50608900199
:107B640070E02434FF22900170E004F080827F00F2
:047B7400227F00224A
:1094B600EFC394339000CB50397431F0EF75F0035D
:1094C600A4241BF582E4340FF583E4939000CCF0DA
:1094D600EF75F003A4241CF582E4340FF583E493BE
:1094E6009000CDF0EF75F003A4241DF582E4340F4F
:1094F600803A7432F075F003EFA4241BF582E5F090
:10950600340FF583E4939000CCF075F003EFA424B8
:109516001CF582E5F0340FF583E4939000CDF075E9
:10952600F003EFA4241DF582E5F0340FF583E493F0
:059536009000CEF022C0
:10B6C400900019E0540F75F00AA4FFA3E0540F2F63
:05B6D40090004CF02283
:10B6D900900019E0540F75F00AA4FFA3E0540F2F4E
:05B6E90090004DF0226D
:10B6EE00900019E0540F75F00AA4FFA3E0540F2F39
:05B6FE0090004EF02257
:10B4660090005EE0FF7E0090005FE0FCA3E0FD122E
:10B476007F0E90005DE02FFF90005CE03EFE9000A6
:0AB4860055E07C002FFFEC3EFE2293
:10B50900303608900037E0FF120086303708900087
:10B5190037E0FF12005E30380D2059FD900037E00A
:07B52900900264F0D25922E8
:10A5B400E4900170F0900047E0FF900170E0FEC36A
:10A5C4009F503F74372EF582E43400F583E0FF900A
:10A5D4000171E4F0A3EFF0303605E0FF120086309D
:10A5E4003708900172E0FF12005E30380D2059FDEB
:10A5F400900172E0900264F0D259900170E004F08E
:03A6040080B322FE
:10AC7000303838E4900170F0900170E0FFC3940424
:10AC8000502974CB2FF582E43400F583E0FF900166
:10AC900071E4F0A3EFF02059FD900172E09002649E
:0CACA000F0D259900170E004F080CD2249
:10ACAC00303838E4900170F0900170E0FFC39405E7
:10ACBC00502974CB2FF582E43400F583E0FF90012A
:10ACCC0071E4F0A3EFF02059FD900172E090026462
:0CACDC00F0D259900170E004F080CD220D
:010078002265
:010079002264
:10AA780030383CE4900170F0900054E0FF90017091
:10AA8800E0FEC39F502974372EF582E43400F58325
:10AA9800E0FF900171E4F0A3EFF02059FD900172FE
:10AAA800E0900264F0D259900170E004F080C9226D
:0C005E0012B69612540712B86102540743
:0C00860012B6AD12540712B86102540704
:10780600E4900170F0900171F0A3F0900173F09094
:1078160000D1E02401FD9000D0E03400FCC3ED94DB
:107826000AEC94005007A3E004900173F0D3ED94A2
:1078360063EC9400405D9000D1E02401FB9000D001
:10784600E03400FA7C007D64AF03FE127F209001D5
:1078560070EFF0E075F064A4FFC3EB9FFFEA95F0CC
:10786600FE7C007D0A127F20900171EEF0A3EFF0FE
:107876009000D1E004FF900170E075F064A4FEC3AF
:10788600EF9EFF900172E075F00AA4FEC3EF9E9092
:107896000173F09000D1E02401FF9000D0E03400A5
:1078A600FED3EF9409EE940040207C007D0A127FFF
:1078B60020900171EEF0A3EFF0E075F00AA4FF90BE
:1078C60000D1E004C39F900173F0900170E0243072
:1078D600F0900172E02430F0900171E03400F090F5
:1078E6000173E02430F030361D900170E0FF120085
:1078F60086900172E0FF120086900173E0FF12008D
:10790600867F2A12008630371D900170E0FF120034
:107916005E900172E0FF12005E900173E0FF1200BC
:077926005E7F2A12005E22C1
:06ABF5007BFF7A127908D3
:10ABFB008B188A19891A20382E7F01127D70E490E8
:10AC0B000170F0900170E0FFC39410501AAB18AABA
:10AC1B0019A91A8F82758300127ECFFF127D3E9089
:08AC2B000170E004F080DC225E
:10A6070090005CF0EFA3F090005E7403F0E490001C
:0AA617005FF0A3F07BFF7A12795880
:10A621008B178A18891920382E7F11127D70E490BA
:10A631000170F0900170E0FFC39410501AAB17AA9B
:10A6410018A9198F82758300127ECFFF127D3E906B
:08A651000170E004F080DC223E
:10B490007BFF7A1279C812A621E4900170F0900126
:10B4A00070E0FF7E00900E9793FD12759F900170E3
:0AB4B000E004F0E0C3940240E5223E
:1093A6007BFF7A1279D812A621E4900173F0E4903B
:1093B6000171F0A3F0E4900170F0900173E075F094
:1093C60099A42402FBE435F0FA900171E0FEA3E0D3
:1093D600FF7C007D03127F0EEF2BFFEE3AFE90011D
:1093E60070E0FD7A002FFFEA3EFEED900E9993FDA8
:1093F60012759F900170E004F0E0C3940340BB90A7
:109406000172E004F07006900171E004F0C390016F
:1094160072E09433900171E094004099900173E0FA
:0994260004F0E0C3941440862216
:109174007BFF7A1279E812A621E4900173F0E4905F
:109184000171F0A3F0E4900170F0900173E0FF7EB0
:10919400007C017D50127F0EEF24F6FBEE340BFAB7
:1091A400900171E0FEA3E0FF1C7D03127F0EEF2B04
:1091B400FFEE3AFE900170E0FD7A002FFFEA3EFEDA
:1091C400ED900E9C93FD12759F900170E004F0E009
:1091D400C3940340B5900172E004F07006900171ED
:1091E400E004F0C3900172E09470900171E0940087
:0F91F4004093900173E004F0E0C3941440802294
:109BB2007BFF7A1279F812A621E4900174F0A3F0E7
:109BC200E4900170F0900170E0FBC39403502E907A
:109BD2000174E0FEA3E0FF7C007D03127F0EEF2400
:109BE20036FFEE3426FEEB2FFFEC3EFEEB900E9F8F
:109BF20093FD12759F900170E004F080C89001758A
:109C0200E004F07006900174E004F0C3900175E086
:0B9C12009488900174E0941340A62297
:01007A002263
:01007E00225F
:01007F00225E
:109C1D007BFF7A13793812A621E4900171F0A3F03D
:109C2D00E4900170F0900170E0FBC39456502E90BB
:109C3D000171E0FEA3E0FF7C007D56127F0EEF2444
:109C4D00CEFFEE3460FEEB2FFFEC3EFEEB900EA54B
:109C5D0093FD12759F900170E004F080C890017221
:109C6D00E004F07006900171E004F0C3900172E021
:0B9C7D009414900171E0940040A622B6
:10B530007BFF7A13794812ABFB12B4901293A612D8
:10B540009174129BB212007A12007E12007F129C3C
:07B550001D127D8D027D9F9D
:10B4BA00E49000D4F0A3F0FFFE1275E09000A8EF2C
:10B4CA00F09000D5E02401FF9000D4E03400FE1291
:08B4DA0075E09000D6EFF022AE
:108AC900756D01756E00756FE9E4900378F0A3F098
:108AD900900378E0FAA3E0FBC39456EA940050406F
:108AE9009000A8E075F056A42478FFE5F03460CF33
:108AF9002BCF3AFE9000D4F0A3EFF01275E0AB6DE6
:108B0900056FE56FAA6E7002056E14F9EF127EFC0F
:108B1900900379E004F070B8900378E004F080B035
:108B2900900116E024FF924B900115E024FF923248
:108B3900900135E0F537900136E0F53890011CE0F9
:108B490024FF924A90011BE024FF923390011AE01E
:108B59007004D2558002C255900113E024FF92237C
:0A8B69009000A974FFF09000AAF03C
:018B730022DF
:10A14000756D01756E01756F48E4900378F0A3F0AA
:10A15000900378E0FEA3E0FFC39414EE9400503B1C
:10A160007C007D56127F0EEF24F9FFEE3460FE90E6
:10A1700000D4F0A3EFF01275E0AB6D056FE56FAAA8
:10A180006E7002056E14F9EF127EFC900379E00404
:0BA19000F070BD900378E004F080B593
:01A19B0022A1
:10A19C00756D01756E01756F5CE4900378F0A3F03A
:10A1AC00900378E0FEA3E0FFC39414EE9400503BC0
:10A1BC007C007D56127F0EEF24FEFFEE3460FE9085
:10A1CC0000D4F0A3EFF01275E0AB6D056FE56FAA4C
:10A1DC006E7002056E14F9EF127EFC900379E004A8
:0BA1EC00F070BD900378E004F080B537
:01A1F7002245
:109203008F17E4900170F0900170E0FBC39403505A
:109213003E9000A8E075F099A42469FDE5F034FFC1
:10922300FCE51775F003A42DFFE5F03CFEEB7C0095
:109233002FFFEC3EFE1275E0900170E024DEF58214
:10924300E43400F583EFF0900170E004F080B8900F
:1092530000DEE0FE54019000D7F0EE54029000D8F7
:10926300F09000DEE054049000D9F0EE5408900032
:10927300DAF09000DEE054109000DBF09000DFE0C5
:0D9283009000DCF09000E0E09000DDF022B3
:109050008F17E4900170F0900170E0FBC39403500F
:10906000449000A8E0FF7E007C017D50127F0EEF4F
:1090700024A6FDEE340AFCE51775F003A42DFFE5E8
:10908000F03CFEEB7C002FFFEC3EFE1275E0900101
:1090900070E024DEF582E43400F583EFF090017097
:1090A000E004F080B29000DEE0FE54019000D7F0C2
:1090B000EE54029000D8F09000DEE054049000D905
:1090C000F0EE54089000DAF09000DEE054109000CA
:1090D000DBF09000DFE09000DCF09000E0E090003A
:0390E000DDF0229E
:068C1A008F178C188D1964
:108C2000E4900378F0A3F0E51924FFFFE51834FF82
:108C3000FE7C007D03127F0EAA06AB07AE17E51778
:108C400025E0CE75F0EEA4FFE5F02EFEEF2448FF00
:108C5000EE3423CF2BCF3AFE900379E02FFF900321
:108C600078E03EFE1275E0900379E024DEF582E4C0
:108C70003400F583EFF0900379E004F07006900380
:108C800078E004F0C3900379E09403900378E094D3
:108C90000040949000DEE0FE54019000E4F0EE54B9
:108CA000029000E5F09000DEE054049000E6F090C1
:0F8CB00000DFE09000E7F09000E0E09000E8F0D7
:018CBF002292
:103D31007BFF7A0079A612ABFB12AE4CE490025FD6
:103D4100F0A3F090017304F0900173E0C394154067
:103D510003023F08900174E4F0A304F0C3900175DD
:103D6100E094FB900174E094004003023EFF900157
:103D710073E0FF7E007C027DEE127F0EEF2448FF90
:103D8100EE342390005CF0FAA3EFF0FB900175E0B4
:103D910024FFFF900174E034FFFE7C007D03127F5D
:103DA1000EEF2BFFEE3AFE1275E0EF54029000DEAB
:103DB100F0900175E024FFFF900174E034FFFE7C78
:103DC100007D03127F0E90005DE02FFF90005CE00C
:103DD1003EFE1275E0EF54049000E1F09000DEE049
:103DE1007003023EEB9000E1E07003023EEB9001B4
:103DF10074E0FEA3E0FF7C007D03127F0E90005D66
:103E0100E02FFF90005CE03ECF24FECF34FFFE1296
:103E110075E09000DFEFF0900174E0FEA3E0FF7C1D
:103E2100007D03127F0E90005DE02FFF90005CE0AB
:103E31003ECF24FFCF34FFFE1275E09000E0EFF09B
:103E4100FD9000DFE0FF125546900171EEF0A3EF07
:103E5100F04E7003023EEB90025FE475F001127FB9
:103E610075AFF0FE900173E0FD12A78890025FE448
:103E710075F001127F75AFF0FE900175E0FD12A79C
:103E81008890025FE475F001127F75AFF0FE90003B
:103E9100DFE0FD12A78890025FE475F001127F75E3
:103EA100AFF0FE9000E0E0FD12A788D3900260E041
:103EB100948890025FE0941340307BFF7A0079B7D9
:103EC10012ABFB90025FE0FEA3E07802CEC313CEFB
:103ED10013D8F9F0EE90025FF09000057414F090A1
:103EE1000005E070030241B980F5900175E004F02E
:103EF1006003023D5D900174E004F0023D5D9001BC
:103F010073E004F0023D49E4900170F0900170E02B
:103F1100FBC3943340030240409000A8E075F09940
:103F2100A42469FDE5F034FFFCEB75F003A42DFF3B
:103F3100E5F03CFE90005CF0A3EFF01275E090001C
:103F4100DEEFF054049000E1F09000DEE0541090B8
:103F510000E2F09000E1E07003024037A3E070035B
:103F610002403790005DE02401FF90005CE03400E6
:103F7100FE1275E09000DFEFF090005DE02402FF9B
:103F810090005CE03400FE1275E09000E0EFF0FD7F
:103F91009000DFE0FF125546900171EEF0A3EFF0C3
:103FA1004E700302403790025FE475F001127F7595
:103FB100AFF0FE7D1512A78890025FE475F0011243
:103FC1007F75AFF0FE900170E0FD12A78890025F4F
:103FD100E475F001127F75AFF0FE9000DFE0FD1295
:103FE100A78890025FE475F001127F75AFF0FE9033
:103FF10000E0E0FD12A788D3900260E0948890026F
:104001005FE0941340307BFF7A0079B712ABFB90ED
:10401100025FE0FEA3E07802CEC313CE13D8F9F01D
:10402100EE90025FF09000057414F0900005E070CE
:10403100030241B980F5900170E004F0023F0DE404
:10404100900170F0900170E0FBC394704003024155
:104051009A9000A8E0FE75F050A4FFE5F02EFEEF67
:1040610024A6FDEE340AFCEB75F003A42DFFE5F068
:104071003CFE90005CF0A3EFF01275E0EF54049069
:1040810000DEF090005CE0FEA3E0FF1275E0EF546B
:10409100109000E1F09000DEE07003024191900089
:1040A100E1E0700302419190005DE02401FF900086
:1040B1005CE03400FE1275E09000DFEFF090005DEF
:1040C100E02402FF90005CE03400FE1275E09000F5
:1040D100E0EFF0FD9000DFE0FF125546900171EE38
:1040E100F0A3EFF09000DEE070030241919000E157
:1040F100E07003024191900171E07002A3E070034E
:1041010002419190025FE475F001127F75AFF0FEFC
:104111007D1612A78890025FE475F001127F75AFDA
:10412100F0FE900170E0FD12A78890025FE475F047
:1041310001127F75AFF0FE9000DFE0FD12A78890BD
:10414100025FE475F001127F75AFF0FE9000E0E0D0
:10415100FD12A788D3900260E0948890025FE094FA
:1041610013402D7BFF7A0079B712ABFB90025FE021
:10417100FEA3E07802CEC313CE13D8F9F0EE90027D
:104181005FF09000057414F0900005E0602A80F85B
:10419100900170E004F002404590025FE0FEA3E070
:1041A1007802CEC313CE13D8F9F0EE90025FF07B04
:0941B100FF7A0079C812ABFB2271
:10A6A800AB07AA067C007D64127F20EF443090003F
:10A6B800CBF07C007D64AF03AE02127F207E007F6A
:10A6C8000ACFCDCFCECCCE127F20EF4430A3F0AE50
:10A6D80002AF037C007D64127F207E007F0ACFCD0D
:0DA6E800CFCECCCE127F20ED4430A3F02267
:10B20C00900022E0540F75F00AA4FDACF0900021E0
:10B21C00E0540F75F064A42DFFE5F03CFE90002384
:10B22C00E0540F7C002FFFEC3EFE900171F0A3EF79
:02B23C00F022FE
:10A560002A2A3132333435362A2A2A2A31323334F0
:10A5700035302A2A44313233343536373839302AA7
:10A580002341424320464C45582049562020412033
:10A59000312E30302020202020534C4156452020A1
:10A5A0002020202020202020204D4153544552209F
:04A5B0002020202027
:1088B600303F23C23F787EE6540F90A57493900113
:1088C6008AF09000077432F09000EAE0601612AD6C
:1088D600D612A818800E900007E07008900176F076
:1088E600900187F0304049C240787CE6540F90A54D
:1088F6007493900189F09000087432F090025EE063
:10890600FF60069000E9E07009EF70099000EBE067
:10891600600312A7D190025EE0FF60069000E9E0D6
:108926007003EF700312AD9B20341312B1A6800EB4
:10893600900008E07008900177F0900186F09002B0
:1089460074E0FF657960149000ECE06018EFD39452
:10895600FA4005E4900274F0027FB1900009E070DD
:0689660004900273F022F0
:10AD9B00900177E0FF04F0EF90A56093FF9001899D
:10ADAB00E0FEEF6E6011EEB42A089001777401F0AB
:10ADBB008005E4900177F0900177E0B40A0C125310
:0BADCB0072E4900177F0D237D24122F1
:10ADD600900176E0FF04F0EF90A56093FF90018A62
:10ADE600E0FEEF6E6011EEB42A089001767401F071
:10ADF6008005E4900176F0900176E0B40A0C1253D7
:0BAE060072E4900176F0D236D24122B7
:10A7D100900186E0FF04F0747D2FF582E43401F5E9
:10A7E10083E0FF900189E0FEEF6E6011EEB4230873
:10A7F1009001867401F08005E4900186F090018655
:10A80100E0B4091212537E125372120056E4900101
:07A8110086F0D237D2352298
:10A81800900187E0FF04F0747D2FF582E43401F5A0
:10A8280083E0FF90018AE0FEEF6E6011EEB423082A
:10A838009001877401F08005E4900187F09001870A
:10A84800E0B4091212537E125372120056E49001BA
:07A8580087F0D236D2352251
:10B1A600900179E0FF04F0EF90A56A93FF90018982
:10B1B600E0FEEF6E6011EEB42A089001797401F09A
:10B1C6008005E4900179F0900179E0B40A04E4F096
:03B1D600D2422240
:10B3B40090017D7423F0A3F0E4FF74ED2FF582E493
:10B3C4003400F583E0FE747F2FF582E43401F583C5
:0CB3D400EEF00FBF06E49001857423F03A
:01B3E000224A
:109FC800127C9B127D8D127D9F7F01127D707BFF1D
:109FD8007AA5798412ABFB90011AE07BFF60067AC0
:109FE800A5799480047AA579A412A6219000057415
:109FF8001EF0E490017BF090017CF0FF74AB2FF52C
:10A0080082E43400F583E4F074BB2FF582E4340075
:10A01800F583E4F00FBF10E4900005E070FA027DCC
:01A028008DAA
:1096B10090017BE0FFD3940F501FEF04FF127D70E8
:1096C100900189E0FF90017BE0FE04F074AB2EF580
:1096D10082E43400F583EF804C7F01127D70E490C9
:1096E1000170F0900170E0FFC3940F5030E0FE2450
:1096F100ACF582E43400F583E0FD74AB2EF582E431
:109701003400F583EDF074AB2FF582E43400F5837A
:10971100E0FF127D3E900170E004F080C690018967
:0A972100E0FF9000BAF0127D3E2236
:1095BB0090017CE0FFD3940F5020EF2411FF127D1C
:1095CB007090018AE0FF90017CE0FE04F074BB2EEA
:1095DB00F582E43400F583EF804C7F11127D70E44B
:1095EB00900170F0900170E0FFC3940F5030E0FEDB
:1095FB0024BCF582E43400F583E0FD74BB2EF582C8
:10960B00E43400F583EDF074BB2FF582E43400F500
:10961B0083E0FF127D3E900170E004F080C6900164
:0B962B008AE0FF9000CAF0127D3E2292
:107FB100900273E0FF702C900274E0FE04F074757F
:107FC1002EF582E43402F583E090017AF090000905
:107FD1007432F090017AE0FEB41B02D241EEB47E1D
:107FE100028064EFB4012A900274E0FF04F074751A
:107FF1002FF582E43402F583E090017AF0900009D4
:108001007432F090017AE0B45002803BE490027344
:10801100F0900273E06402703A900274E0FF04F0A1
:1080210074752FF582E43402F583E090017AF090C3
:1080310000097432F09000D6E075F00A844430FFF4
:1080410090017AE0B50707900273E004F022E49012
:108051000273F0900273E064037044900274E0FFD5
:1080610004F074752FF582E43402F583E090017A0F
:10807100F09000097432F0E4900273F09000D6E0C1
:1080810075F00A84E5F04430FF90017AE0B5070FFE
:10809100E4900014F0D238D235D239C250C2512204
:105D9200755900125DAD50FB22755900125E3650E6
:105DA200FB22755900125DED50FB22758400E55906
:105DB20075F003A4905DBA73025E52025E61025EE8
:105DC2007F025E68025E8B025E92025E9A025E61F2
:105DD200025EA8025E68025EB8025EC1025E520204
:105DE2005E61025ECF025E68025EDB758400E55989
:105DF20075F003A4905DFA73025E52025E61025E68
:105E02007F025E68025E8B025E92025E52025E61F9
:105E1200025E7F025E68025E8B025E92025E8B020F
:105E22005E92025E9A025E61025EDD025E68025E60
:105E3200B8025EDB758400E55975F003A4905E43F9
:105E420073025E52025E61025ECF025E68025EDB38
:105E5200C2FA125EED125EED759B000559C3223047
:105E6200F9020559C32230F912E59A20E7FB125EC6
:105E7200EDD2FA125EED125EED0559C322C2FA129C
:105E82005EED759B040559C32275411E0559C32257
:105E9200E54170020559C322C2FA125EED125F0E8D
:105EA200F59B0559C322C2FA125EED125F1D44072B
:105EB200F59B0559C322125EFFF5420559C32275AF
:105EC200840F30DE04E54270020559C322C2FA1281
:105ED2005EED759B080559C322D322C2FA125EED0C
:095EE200125F1D4405F59B0559F2
:105EEB00C3220000000000000000000000000000C2
:105EFB0000000022905F06E55A93225A5A5A5A5ACA
:105F0B00FAFAFA905F15E55A932200B45AE12D87FD
:105F1B007ADB905F24E55A9322000000000000809A
:015F2B0080F5
:1013E800C0D0C000C001C083C082C0E0C0F0C00748
:1013F800A292304B01B3787BE233F208E233F20871
:10140800E233F208E233F208E233F208E233F20898
:10141800E233F208E233F208E233F208E233F20888
:10142800E233F208E233F208E233F208E233F20878
:10143800E233F208E233F208E233F208E233F20868
:10144800E233F208E233F208E233F208E233F20858
:10145800E233F208E233F208E233F208E233F20848
:10146800E233F208E233F208E233F208E233F20838
:10147800E233F208E233F208E233F208E233F20828
:01148800E281
:1014890033F208E233F208E233F208E233F208E217
:1014990033F208E233F2305C359018B478A2E218DE
:1014A900202303936028E218937023E21893601EA7
:1014B900E218937019E218936014E21893600FE22E
:1014C9001893700AE218937005E2189360030216E4
:1014D9008E755000E2189313924350037550387576
:1014E9002300E2189313921C500363501CE21893D3
:1014F90013921B500363500EE2189313921A500370
:10150900635046E218931392195003635023E2186B
:10151900931392188523515003635051752300E2A8
:10152900189313921C5003635068E2189313921B8B
:101539005003635075E2189313921A500363507A5B
:10154900E21893139219500363503DE218931392D2
:1015590018852352500363501F752300E218931313
:10156900921F500363504FE2189313921E50036366
:101579005026E2189313921D5003635052E21893B8
:1015890013921C5003635029E2189313921B5003C2
:10159900635015E2189313921A500363500BE21823
:1015A900931392195003635045E2189313921885C7
:1015B90023535003635062E2189313921C50036340
:1015C9005031E2189313921B5003635019E2189398
:1015D90013921A500363500DE21893139219500392
:1015E900635007E2189313921885235450036350EC
:1015F90043752300E2189313921EE2189313921D68
:10160900E2189313921CE2189313921BE218931396
:10161900921AE21893139219E218931392188523D8
:1016290055C248E55565506035D24823F8901E05E6
:1016390093F9901E04E8936025B40104B243801E17
:0E164900B40205E862518016B40305E862524F
:10165700800EB40405E862538006B4052AE8625494
:10166700A24392449000A3E551F09000A4E552F004
:101677009000A5E553F09000A6E554F0304706D258
:1016870046C2478002D2471216A2D007D0F0D0E058
:10169700D082D083D001D000D0D022C0D0C000C02B
:1016A700E0302D4EE562B40833A230B392B37880B0
:1016B700E66036167885E6A2E7303201B3923092BB
:1016C700B2A2E77881E633F67882E633F67883E6E6
:1016D70033F67884E633F67885E633F6D562037514
:1016E7006208D0E0D000D0D022C254D0E0D000D0E1
:1016F700D022D0E0D000D0D022C0D0C000C001C0DE
:1017070083C082C0E0C0F0A292204A01B37863E2AE
:1017170013F208E213F208E213F208E213F208E206
:1017270013F208E213F208E213F208E213F208E2F6
:0D17370013F208E213F208E213F208E213C5
:10174400F208E213F208E213F208E213F208E213D9
:10175400F208E213F208E213F208E213F208E213C9
:10176400F208E213F208E213F208E213F29018B45A
:101774007863E20893139217E20893139216E2082F
:1017840093139215E20893139214E208931392139D
:10179400E20893139212E20893139211E20893134E
:1017A4009210852256E20893139217E2089313923B
:1017B40016E20893139215E20893139214E2089325
:1017C400139213E20893139212E20893139211E214
:1017D4000893139210852257E20893139217E20894
:1017E40093139216E20893139215E208931392143A
:0117F400E212
:1017F5000893139213E20893139212E2089313923B
:1018050011C210852258305C3DE556901C04855761
:1018150022301602058393602D14F875F003A49009
:101825001AB52582F582E5F03583F583E493F9A3AE
:10183500E4939019B4655893C965579329B4010089
:1018450050048844D22F12185DD0F0D0E0D082D059
:1018550083D001D000D0D022302B26788616E670B2
:101865002076087889E6A2E1303301B392B292B3CB
:10187500A2E17887E613F67888E613F67889E61309
:10188500F622EF901AB475F003A42582F582E5835C
:1018950035F0F583C22B7400937887F6740193783D
:1018A50088F67402937889F6C22DC22CD22B2200B9
:1018B5000000000000000000000000000000000023
:1018C5000000000000000000000000000000010012
:1018D5000000000000000000000000000000010002
:1018E50000000000000001000000010001010100EE
:1018F50000000000000000000000000000000100E2
:1019050000000000000001000000010001010100CD
:1019150000000000000001000000010001010100BD
:1019250000000100010101000101010101010100A7
:1019350000000000000000000000000000000100A1
:10194500000000000000010000000100010101008D
:10195500000000000000010000000100010101007D
:101965000000010001010100010101010101010067
:10197500000000000000010000000100010101005D
:101985000000010001010100010101010101010047
:101995000000010001010100010101010101010037
:1019A5000101010101010101010101010101010023
:1019B5000101020102020301020203020303040101
:1019C50002020302030304020303030303040501E4
:1019D50002020302030304020303040304040502D1
:1019E50003030403040405030404040405050601B4
:1019F50002020302030304020303030304040502B2
:101A05000303040303040503040405040505060292
:101A15000303040304040503040405040505060380
:101A25000404050405050604050506050606070163
:101A35000202030203030402030304030404050270
:101A45000303040304040503040405040505060251
:101A55000303040304040503040405040505060340
:101A65000404050405050604050506050606070222
:101A75000303040304040503040405040505060320
:101A85000404050405050604050506050606070301
:101A950004040504050506040505060506060704F0
:101AA500050506050606070506060706070708FDD8
:101AB500D00C73700E3CF01AAF101E7F9022EC70A4
:101AC50026D6F02ACBB02CA3F032BEB03417D03CCA
:101AD500B6D0461FB04E77F050F950526AB056DE78
:101AE5009058BA306ACF3072D270745CD076E8F014
:101AF500786BD098E5709AF8309CBB50A40F70AA0B
:101B05007A70B26730B45DB0B8FCB0C26F50C655DC
:101B1500D0CA3D90D489B0DA94F0DCD790E463B0B4
:101B2500EA0BF0F43170F8DD310AB571148FF11854
:101B3500D1D126EB512AF6112C8B71463F5148B174
:101B4500F14AACB14CC4F152D9B1546D915A2EF150
:101B550062BD116687916A9AD16CF29172D55178FE
:0D1B650019F18C71B192D8D19A32D1AA47F2
:101B7200D1B25A91B452F1C67531CC1D71D2A9516C
:101B8200DCD0B1E85E11EA2B11F2EED212F392141C
:101B92007D3216973226D8B232C5F234F7124AEAAB
:101BA200524C9F5254A5D2582B725A7552644FD23E
:101BB20068C1726ADC326C78D2865F128C83729C46
:101BC2004EB2A66972AC1C72B433D2CC18F2EABB24
:101BD200330CCE33141EB32803F32EE51332F8531D
:101BE2003498735848F36472736845738617B394D4
:101BF2007313A63C93B221D3B41B53B829B3C64185
:101C0200F3D8000000000000000000000000000007
:101C12000000000000000000006A00000000000058
:101C2200620D0000000000000000006F004800008C
:101C320000000000000000000000000000006C2214
:101C42000000000000000000000000000000000092
:101C52005B00000000000000000000004100001EC8
:101C62004759000000260000001D0000100000354A
:101C72000000003D006B0043000000000000004B2C
:101C820000050000000000000038002300000000F2
:101C92000000000000000000004C000000000000F6
:101CA2000000000000000000000000000000320000
:101CB2000004000000000000000000001260003775
:101CC2000A00000000000000000000000008000000
:101CD200611346000000000000254D340000572922
:101CE200110000000000006400000000000000007D
:101CF200000000003A4A00002E4F190000001F00A9
:101D02000000000000630000000000000027000047
:101D1200001B000000000000000B5F3C006E5D44F1
:101D22000000006D000000000000000000530000F1
:101D3200360000283F5E00000000000000000300A3
:101D420000300070000000690040670000000000E1
:101D520000550000420000210000000000001500B4
:101D620000000000000000000000005C00170000FE
:101D72000020000068020054000E58001C00000001
:101D820000000000005A000000000000002F0000C8
:101D9200002B000000002400000066003900000053
:101DA2000051000000090052000000450000000040
:101DB200000000310000002A0C000000001A0000A0
:101DC200000000560000334E00000000000000003A
:101DD2000000002C1400003B07003E000000000041
:101DE200000000000000001800001600502D060040
:101DF20049000000000000000000650F0000000123
:101E020000000000000000000600000006000600BE
:101E12000502060006000600040406000504020886
:101E22000600000006000600060006000408060080
:101E3200060006000508060006000210060006005D
:101E4200030100000600060002020600060004402C
:101E52000600060004100600060006000600060042
:101E62000600060005100600060006000600060031
:101E72000600010106000600060006000302060035
:101E82000600000006000600050106000402020426
:101E92000600060006000600060006000600060010
:101EA2000480060002010420060006000600060067
:101EB20006000600060006000600060006000600F0
:101EC20006000600060004010600060006000600E1
:101ED20006000310060006000600060006000600C3
:0D1EE20006000600060006000600060003CC
:101EEF0008060006000600060003040600060006AA
:051EFF000006000600D2
:1048E200758400C2CA85CC4885CD4775CC0075CD8C
:1048F20000D2CA10CF02D25B32305B0BC25BE547FB
:10490200C3943640028001227891798F7B06E7F6C4
:104912001819DBFAA64718A648AA48AB47AE02AF59
:1049220003EEC4035407FEEFC403FF54F84EFEEF38
:104932005407FF7803798CC3E79AFC09E79BFD09CA
:1049420050066304FF6305FFC3EC9EED9F5074D8CD
:10495200E6789979977C06E7F61819DCFAA6031827
:10496200A6027994AE02AF03EEC423541FFEEFC435
:1049720023FF54E04EFEEF541FFF7803C3E79AFC77
:1049820009E79BFD0950066304FF6305FFC3EC9E24
:10499200ED9F502FD8E678927A007B007C00790454
:1049A200EA26FA08EB36FB08EC3400FCD9F2EC13E9
:0D49B200FCEB13FBEA13FAEC13EB13F546D4
:1049BF00EA13F545D22122302131C2211249FB5091
:1049CF002A854C4D854B4C854A4B85494A8507496D
:1049DF00302013E54F6F600EE507B54A0EB54B0B50
:1049EF00B54C08B54D0585074ED22222904B16E5E2
:1049FF004693FF904A4223232582F582E5833400B4
:104A0F00F583124A21400A0F124A2140040F124A1D
:104A1F002122E493F9A3E493FAA3E493FBA3E49391
:104A2F00FCA3C3E5459AE546995007C3EC9545EBC2
:104A3F00954622EA25DD89DD89D324D324CBD2CB39
:104A4F00D2C4DBC4DBBE39BE39B7CAB7CAB18EB167
:104A5F008EAB87AB87A59CA59CA000A0009A969AC9
:104A6F009695D895D891E591E58D858D8588AF88F8
:104A7F00AF840C840C7F9A7F9A7B497B49771B7795
:104A8F001B730F730F6F276F276B576B5767AB67CF
:104A9F00AB642C642C60C660C65D795D795AFE5A92
:104AAF00FE5970597057E257E25661566154E754F8
:104ABF00E7537453745207520750A050A04F404F02
:104ACF00404DE64DE64C934C934B414B4149F549D4
:104ADF00F548B548B547764776463E463E450845C4
:104AEF0008432A432A40E440E43F533F533E3E3EAF
:104AFF003E3C943C943A863A86391839183805006A
:104B0F0000000000000000323232323232323232D4
:104B1F003232323232323232323232323232323266
:104B2F003232323232323232323232323232323256
:104B3F003232323232323232323232323232323246
:104B4F00313130302F2E2D2D2D2C2C2B2A29292889
:104B5F0027262525242323222120201F1E1E1D1C2E
:104B6F001C1B1A1A1A1A19191918181817171717A8
:104B7F0016161616151515151414141413131313DE
:104B8F00121212121111111110101010100F0F0F0D
:104B9F000F0F0E0E0E0E0D0D0D0D0C0C0C0C0B0B36
:104BAF000B0B0B0B0A0A0A0A0A090909090909085A
:104BBF000808080808070707070707060606060676
:104BCF00060605050505050504040404040404038D
:104BDF0003030303030302020202020202010101A3
:104BEF0001010101010101010101010000000000AB
:104BFF0000000000000000000000000000000000A6
:104C0F0000000000000000302C0D852F8A852E8CAF
:0A4C1F00D28CB2B1D2A932C28C22AD
:10706B00C007C0007F01127D707F4C127D3E7F54A4
:10707B00127D3E7F52127D3E7F20127D3E204404C6
:10708B007F3080027F31127D3E7F20127D3E90004B
:10709B00A4E0785D1254DA785D8607430730127DE1
:1070AB003E088607430730127D3E750720127D3E52
:1070BB009000A5E0785D1254D2785D8607430730C7
:1070CB00127D3E088607430730127D3E0886074334
:1070DB000730127D3E750720127D3E9000A3E078AD
:1070EB005D1254DA785D8607430730127D3E0886C1
:1070FB0007430730127D3E750720127D3ED000D02E
:10710B000722C007C0007F11127D707F4C127D3E9D
:10711B00750720127D3E2049047F3080027F31129B
:10712B007D3E7F20127D3E9001F9E0785D1254DAAE
:10713B00785D8607430730127D3E0886074307308C
:10714B00127D3E750720127D3E9001FAE0785D12AC
:10715B0054D2785D8607430730127D3E088607437D
:10716B000730127D3E088607430730127D3E7507B8
:10717B0020127D3E9001FBE0785D1254DA785D863B
:10718B0007430730127D3E088607430730127D3ECA
:10719B00750720127D3E9001FCE0785D1254DA7881
:1071AB005D8607430730127D3E0886074307301282
:0771BB007D3ED000D0072249
:106AF600003800512372461765340E5F2D7C481905
:106B06006B3A1C4D3F6E5A0B79281243316054057F
:106B16007726001F3D227A654758756A48570F1039
:106B2600322D6877554A120D2F301D02203F6778A7
:106B36005A45006245270B694E2C157750321E7C4C
:106B46005B39294B6C0E224067053C5E791B375535
:106B5600721052301775593B1C7E472502604C2E29
:106B6600096B7B193E5C701235576E0C2B49650715
:106B76002042264463012D4F680A33517614385A51
:106B86007D1F0F6D4A28046641231A785F3D1173F5
:106B96005436741631537F1D3A58610324466A08E9
:106BA6002F4D5D3F187A56341371482A0D6F4321D5
:106BB60006644F2D0A68442601635A381F7D5133F7
:106BC6001476660423416D0F284A73113654781AD9
:106BD6003D5F1D7F583A16745331086A4D2F036185
:106BE6004624345671133F5D7A18214364062A48B9
:106BF6006F0D690B2C4E620027457C1E395B77159D
:106C06003250402205674B290E6C553710725E3C98
:106C16001B793B597E1C305275172E4C6B09254744
:106C2600600212705735197B5C3E076542200C6E78
:106C3600492B004307440D4E0A49195A1E5D145745
:106C46001350317236753C7F3B78286B2F6C256666
:026C56002261B9
:108D5D00788576ACA249E433FFC4333354C0FE901A
:108D6D0001FBE0FD541F25E04EFE9001F9E0FC549F
:108D7D0010C4540F4E7884F6EC540FC454F0FE908A
:108D8D0001FAE0FC54F0C4540F4E7883F6EC540F06
:108D9D00C454F0FE9001FCE0FC541EC3134E7882C7
:108DAD00F6EF3395E0FE74F62FF582746A3EF58387
:108DBD00E493FFED906AF893FEEF6EFF9001F9E0FA
:108DCD00906B18936FFF9001FAE0906B38936FFFE3
:108DDD00EC906C38936F7881F69001FCE030E004F4
:0B8DED00E64480F6D2547880762822FD
:10A50B00758401309914C299204C0F9001F7E070BB
:10A51B0009D24CD29C789A7604223098379001F865
:10A52B00E06401702DE55B75F00584205211248DDC
:10A53B00F582E43401F583E599F0C298D2522224D6
:10A54B00A2F582E43401F583E599F0C298C252D2A8
:05A55B005322C298220A
:108337007584012098030283FD204E13209A0DE5D2
:10834700997009D24ED24F755C0AF55BC29822909C
:1083570001F8E0FF6401702CE55B75F0058420529D
:1083670010248DF582E43401F583E599F0D252802B
:108377001024A2F582E43401F583E599F0C252D2C4
:1083870053C29822EFB4021AAB6D056FE56FAA6E60
:108397007002056E14F9E599127EFC9001F87403DA
:1083A70080209001F8E0FFB4031CAB6D056FE56F0B
:1083B700AA6E7002056E14F9E599127EFC9001F819
:1083C7007404F0C29822EFB4042990022AE0FF0453
:1083D700F074012FF582E43402F583E599F0C29831
:1083E70090022AE0B4281C90022C7401F0E490015A
:1083F700F8F022C2982230990AC2999001F7E070EA
:0484070002C2522239
:10B55700204D2212539743E740755C0AE4F55B9050
:10B5670001F7F09001F8F0C24CD24D75840175983F
:06B5770090C29CF5992230
:109F650090022BE0705C90036FE0FF7025D39001A9
:109F7500FEE094869001FDE094674008E4F0A37448
:109F850002F0800E9001FEE02428F09001FDE034FF
:109F950000F09001FEE02FFF9001FDE03400FE127D
:109FA50075E090036FE02401F582E43402F583EF58
:109FB500F090036FE004F0E0B42807E4F090022B82
:039FC50004F02283
:1090E30090022CE070030291739001FFE0FEA3E075
:1090F300FFC39402EE94005006E490022CF02290F9
:10910300036FE07C002FFFEC3EFE1275E090036FCF
:10911300E02401F582E43402F583E0FD6F601790EB
:10912300036FE0FF900200E02FFF9001FFE03400A7
:10913300FE12759FD25090036FE004F0E064287034
:109143002F90022CF090036FF09001FFE0FEA3E05C
:10915300FFBE2008BFD205E490036FF0EF64024E18
:10916300700E30500BC250128AC912A14012A19C3A
:0191730022D9
:109E2F00304C6475840190023EE0B40D00505590A3
:109E3F009E45F8282873029E6C029E6F029E720246
:109E4F009E75029E78029E7B029E7E029E81029EDE
:109E5F0084029E87029E8A029E8D029E9002B358B4
:109E6F0002B70302A92C02ACE802B5C602001E021B
:109E7F00B1D902B00C02AD2402A96F02B66402B4CC
:089E8F000E02B64912B67E2254
:10B35800789AE67028759898755C0AF55B9000A84D
:10B36800E0B4010790023E7404F022E49001F8F082
:0EB378009001F7F090023EE004F01253942290
:10B703009001F87401F0E49001F7F0C25290023E08
:04B71300E004F0223C
:10A92C009000A8E01475F005A4B55B19E4B5F0151A
:10A93C00759898125397E49001F7F09001F8F09005
:10A94C00023E7404F0E55B75F00584AFF0BF0112B4
:10A95C00C253E49001F7F09001F804F090023EE04D
:03A96C0004F022D2
:10ACE800E55B75F00584AFF0BF043020531EE55BCB
:10ACF80075F00584FF248DF582E43401F583E4F0D2
:10AD080074A22FF582E43401F583E4F0E49001F7AE
:0CAD1800F09001F8F090023EE014F022F0
:10B5C6009000A8E075F005A424FDB55B159000A9D0
:10B5D600E0F599E49001F7F09001F8F090023EE072
:03B5E60004F0224C
:0D001E009000AAE0F59990023EE004F02267
:10B1D9009000A8E0FD75F005A4FFE55BB50723E441
:10B1E900B5F01FEDB4140790023E7409F022125312
:10B1F90094E49001F7F0C2529001F8F090023EE019
:03B2090004F0222C
:10B00C00E55BB46412125397E49001F7F09001F8E9
:10B01C00F090023E7409F0E55B75F00584AFF0BF6B
:10B02C000112C253E49001F7F09001F804F0900281
:05B03C003EE004F022DB
:10AD2400E55B75F00584AFF0BF043020531EE55B8E
:10AD340075F00584FF248DF582E43401F583E4F095
:10AD440074A22FF582E43401F583E4F0E49001F772
:0CAD5400F09001F8F090023EE014F022B4
:10A96F00E55B6465703C90022BE0B4012F756D01BF
:10A97F00756E01756FFDE49001F7F09001F8F075B9
:10A98F008401AB6D056FE56FAA6E7002056E14F949
:10A99F00127EB6F59990023EE004F02290023E74CA
:03A9AF000CF02287
:10B66400758401AB6DAA6EA96F127EB6F599E4904C
:0AB674000229F090023EE004F022EB
:10B40E00758401900229E0FF04F074012FF582E4A7
:10B41E003402F583E0F599900229E0D39428400B8D
:0CB42E00E490022BF090023EE004F022BB
:10B64900E55BB46915C24CC24DE490018BF09001E1
:0BB65900F7F09001F8F090023EF022A4
:10B67E00C24CC24DE4F55B90018BF09001F7F09057
:08B68E0001F8F090023EF022E9
:10A3B600304E5275840190023FE0B40A005043903B
:10A3C600A3CCF828287302A3EA02A3ED02A3F002A5
:10A3D600A3F302A3F602A3F902A3FC02A3FF02A4BD
:10A3E6000202A40502AFD602AEBF02AF3002B62A01
:10A3F60002B78502B43A02AA3702AF6802B60A0269
:06A40600B76412B79522B5
:10AFD600E55B70317598989000A8E0B401131253A0
:10AFE60097E49001F8F09001F7F090023F7403F0B7
:10AFF60022125394C252E49001F8F09001F7F090B7
:06B00600023FE004F0220D
:10AEBF009000A8E01475F005A4B55B11E4B5F00D92
:10AECF0075989812539790023F7403F022E55B75C3
:10AEDF00F00584AFF0BF0110C253C2529001F87455
:09AEEF0001F090023FE004F022A2
:10AF3000E55B75F00584AFF0BF042C20531EE55B84
:10AF400075F00584FF248DF582E43401F583E4F087
:10AF500074A22FF582E43401F583E4F0E49001F863
:08AF6000F090023FE014F02222
:10B62A009000A8E075F005A424FDB55B11758401AE
:0FB63A009000A9E0F599C25290023FE004F0227F
:10B785007584019000AAE0F59990023FE004F0224B
:10B43A009000A8E0FFB4140790023F7406F022EFD0
:10B44A0075F005A4B55B14E4B5F01012539490029C
:0CB45A003FE004F0C252E49001F8F02240
:10AA3700E55B75F00584AFF0BF0111C253C25290B8
:10AA470001F87401F090023FE004F022E55BB46482
:10AA57001F12539490022CE0700B9001F8F09002B3
:10AA67003F7408F022E49001F8F090023F7409F077
:01AA770022BC
:10AF6800E55B75F00584AFF0BF042C20531EE55B4C
:10AF780075F00584FF248DF582E43401F583E4F04F
:10AF880074A22FF582E43401F583E4F0E49001F82B
:08AF9800F090023FE014F022EA
:10B60A00E55BB4651A756D01756E01756FFFE4909F
:10B61A00022AF090023F7409F09001F87402F022B5
:10B76400E55BB4690BC24EE49001F8F090023FF03F
:01B7740022B2
:10B79500C24EE49001F8F09001F7F090023FF022DC
:10745F00789DE660011678A3E6600116900000E0C3
:10746F00600214F0900002E0600214F0900001E05E
:10747F00600214F0900003E0600214F0900004E04A
:10748F00600214F0900010E0600214F090000FE022
:10749F00600214F0900253E0600214F090025CE07E
:1074AF00600214F0789F16E6600302759E789F764F
:1074BF000A789EE6600116E54260021542900005CB
:1074CF00E0600214F0900006E0600214F0900007F4
:1074DF00E0600214F0900008E0600214F0900009E0
:1074EF00E0600214F090000AE0600214F090000BCC
:1074FF00E0600214F090000DE0600214F090000EB6
:10750F00E0600214F0900256E0600214F078A4E6F6
:10751F0060011690026CE0600214F090026FE06060
:10752F000214F0900270E0600214F078A016E6707A
:10753F005E78A0760A900012E0600214F078A6E65A
:10754F001846600708E6161870011690025DE06095
:10755F000214F090025EE0600214F090026AE060A4
:10756F000214F0900272E0600214F078A116E67037
:10757F001E78A1760A900013E0600214F078A2162C
:10758F00E6700C78A27606900011E0600214F022EB
:1080A100535155452020434F53202053454E5345AE
:1080B100004F4E2020202020202020202020202082
:1080C10020004F4646202020202020202020202054
:1080D100202000242424242424242424242424248B
:1080E100242424242424242424242424242424244F
:1080F100242424242424242424242424242424243F
:10810100242424231A1B1C1D1E1F20212224242465
:1081110024242424000102030405060708090A0B8C
:108121000C0D0E0F10111213141516171819242403
:1081310024242424000102030405060708090A0B6C
:108141000C0D0E0F101112131415161718192424E3
:1081510024242400000AAB0D55100012AB1555184C
:10816100001AAB1D55200022AB255528002AAB2D46
:0D81710055300032AA355538003AAA3D5568
:10B57D00751F01E51FC394155018AF1F74B62FF535
:10B58D0082E43401F583E0FFEF60037F0122051FA4
:04B59D0080E17F00CA
:01B5A1002287
:10A30700205455128675EF6401704D900119E0FFD6
:10A31700EF24FF92499001F6E0FF74E02FF582E405
:10A327003401F583E0FF9001F9EFF09001F6E0FFCB
:10A3370074CB2FF582E43401F583E0FF9001FAEF47
:10A34700F09001F6E0FF9001FBEFF0125702900149
:09A35700FCEFF0128D5DD22D2205
:10867500900171E4F0A3E4F0900174E4F0A3E4F058
:10868500900170E4F0900170E0FFEFC39415400392
:108695000287199001F6E0FFEFD39414400690018C
:1086A500F67401F09001F6E0FF74B62FF582E4341C
:1086B50001F583E0FF900173EFF0900173E0FFEFA8
:1086C500B401159001F6E0FF74B62FF582E434018C
:1086D500F5837402F07F0122900173E0FFEFB4028D
:1086E50024900171E0FEA3E0FFEF4E701890017138
:1086F500E4F0A37401F09001F6E0FF7E00900174B0
:10870500EEF0A3EFF09001F6E004F0900170E004C4
:10871500F002868A900171E0FEA3E0FFEF4E70043F
:108725007F002222900175E0FF9001F6EFF07F01B6
:018735002221
:1084DD00900171E4F0A3E4F0900174E4F0A3E4F0F2
:1084ED00900170E4F0900170E0FFEFC3941540032C
:1084FD0002858E9001F6E0FFEFD3941440069001B3
:10850D00F67401F09001F6E0FF74B62FF582E434B5
:10851D0001F583E0FF900173EFF0900173E0FFEF41
:10852D0060509000A8E0FF9001F6E0FEEE6F604213
:10853D00900173E0FFEFB401159001F6E0FF74B602
:10854D002FF582E43401F5837402F07F012290014E
:10855D0071E0FEA3E0FFEF4E70189001F6E0FF7E94
:10856D0000900174EEF0A3EFF0900171E4F0A374AC
:10857D0001F09001F6E004F0900170E004F0028447
:10858D00F2900171E0FEA3E0FFEF4E70047F002238
:0E859D0022900175E0FF9001F6EFF07F0122C1
:105702009000A8E0FFEFD3941440037F202290037F
:1057120073E4F0900372E4F09000A8E0FF9003704D
:10572200EFF0900114E0FFEFD3940650030257F616
:10573200900371E4F0900371E0FFEFC3941540030E
:105742000257EF900370E0FFEFB4150690037074F8
:1057520001F0900370E0FF748C2FF582E43401F5C0
:1057620083E0FFEF64FF7076900370E0FF74472FD1
:10577200F582E43401F583E0FF9000A8E0FE74476F
:105782002EF582E43401F583E0FEEEC39F404F9094
:1057920000A8E0FF900370E0FEEEB50706900370EC
:1057A200E0FF22900370E0FF74472FF582E434019A
:1057B200F583E0FF900372E0FEEFD39E402090035A
:1057C20070E0FF900373EFF0900370E0FF74472FD7
:1057D200F582E43401F583E0FF900372EFF0900369
:1057E20071E004F0900370E004F002573790037305
:1057F200E0FF2222900371E4F0900371E0FFEFC317
:10580200941540030258B2900370E0FFEF700690C7
:1058120003707414F0900370E0FF748C2FF582E42F
:105822003401F583E0FFEF64FF7076900370E0FFD0
:1058320074472FF582E43401F583E0FF9000A8E07D
:10584200FE74472EF582E43401F583E0FEEEC39F39
:10585200404F9000A8E0FF900370E0FEEEB507060F
:10586200900370E0FF22900370E0FF74472FF582EF
:10587200E43401F583E0FF900372E0FEEFD39E4033
:1058820020900370E0FF900373EFF0900370E0FF4D
:1058920074472FF582E43401F583E0FF900372EF41
:1058A200F0900371E004F0900370E014F00257FBF3
:0558B200900373E0FF0C
:0158B70022CE
:1058B8009000A8E0FFEFD3941440037F20229003C8
:1058C80077E4F0900376E4F0900114E0FFEFD394CE
:1058D80006500302599D9000A8E0FFEF04FF9003D3
:1058E80074EFF0900375E4F0900375E0FFEFC39454
:1058F800154003025996900374E0FFEFD3941440C7
:10590800069003747401F0900374E0FF748C2FF513
:1059180082E43401F583E0FFEF64FF706290037462
:10592800E0FF74472FF582E43401F583E0FF90002F
:10593800A8E0FE74472EF582E43401F583E0FEEE1C
:10594800C39F403B900374E0FF74472FF582E43413
:1059580001F583E0FF900376E0FEEFD39E402090B0
:105968000374E0FF900377EFF0900374E0FF74474F
:105978002FF582E43401F583E0FF900376EFF09091
:105988000375E004F0900374E004F00258F090030B
:1059980077E0FF22229000A8E0FFEF14FF90037445
:1059A800EFF0900375E4F0900375E0FFEFC39415F2
:1059B8004003025A52900374E0FFEF70069003749C
:1059C8007414F0900374E0FF748C2FF582E43401B2
:1059D800F583E0FFEF64FF7062900374E0FF7447A3
:1059E8002FF582E43401F583E0FF9000A8E0FE740F
:1059F800472EF582E43401F583E0FEEEC39F403B79
:105A0800900374E0FF74472FF582E43401F583E0D6
:105A1800FF900376E0FEEFD39E4020900374E0FFF2
:105A2800900377EFF0900374E0FF74472FF582E45A
:105A38003401F583E0FF900376EFF0900375E004FE
:0F5A4800F0900374E014F00259AF900377E0FF81
:015A5700222C
:10B717009000A8E0FFEFD3941440037F202290000D
:04B72700A8E0FF2275
:1076D8009001F5E0FFEFD3941440069001F5740192
:1076E800F0900170E4F09001F5E0FF74CB2FF58283
:1076F800E43401F583E0FF9001F5E0FE74A12EF576
:1077080082E43401F583E0FEEEB507269001F5E04A
:10771800FF74E02FF582E43401F583E0FF9001F572
:10772800E0FE748C2EF582E43401F583E0FEEE6F02
:1077380060069001707401F09001F5E0FF748C2FE1
:10774800F582E43401F583E0FF9000A8E0FEEF6ED7
:10775800600E9000A8E0FF9001F5E0FEEE6F703A31
:10776800900170E0FFEF60439001F5E0FFEFD394E4
:107778001550149001F5E0FF74B62FF582E434013A
:10778800F5837401F080249001F5E0FF74B62FF5BD
:1077980082E43401F583E4F080119001F5E0FF7490
:1077A800B62FF582E43401F583E4F0900170E0FF30
:1077B800EF60449001F5E0FF74A12FF582E43401F5
:1077C800F583E0FF9001F5E0FE74CB2EF582E434FA
:1077D80001F583EFF09001F5E0FF748C2FF582E45A
:1077E8003401F583E0FF9001F5E0FE74E02EF582A8
:0E77F800E43401F583EFF09001F5E004F02297
:106C5800900239E0FFEF6003026D1390000BE0FF34
:106C6800EF70037F012212A9F5EFB4010312009619
:106C780012A9F5EF70031200562046037F00221276
:106C8800A9F5EF64016003026D1330467BC246200C
:106C9800360920370620380312706B9000A4E0FFF5
:106CA800900235EFF09000A5E0FF900236EFF090EB
:106CB80000A3E0FF900237EFF0900237E0FFEFB457
:106CC8001F14900233E0FF900236E0FEEEB507068F
:106CD8001200567F0122900232E0FF900235E0FE5A
:106CE800EEB5070E900233E0FF900236E0FEEE6F3D
:106CF80060099002397401F07F002290010BE0FFD7
:106D080090000BEFF07F00227F0022900239E0FF15
:106D1800EF64016003026DB590000BE0FFEF7003B4
:106D28007F012212A9F5EFB4010312009612A9F50A
:106D3800EF70031200562046037F0022C2461270ED
:106D48006B9000A4E0FF900235EFF09000A5E0FF03
:106D5800900236EFF09000A3E0FF900237EFF0903A
:106D68000237E0FFEFB41F14900233E0FF900236C1
:106D7800E0FEEEB507061200567F0122900232E0CF
:106D8800FF900235E0FEEEB50720900233E0FF9059
:106D98000236E0FEEEB5071290010BE0FF90000B03
:106DA800EFF0900239E4F07F00227F00227F00227A
:10A9F500900102E0FFEF600D12539A40047F018041
:10AA0500027F002222900103E0FFEF601390010412
:10AA1500E0FFE532D39F40047F0122227F002222FE
:10AA2500900104E0FFE532C39F50047F0122227F9D
:02AA35000022FD
:109DC600900170E4F0900170E0FFEFC3940A5058E0
:109DD600900170E0FF74262FF582E43401F583E0EC
:109DE600FFEFB42013900170E0FF743E2FF582E47C
:109DF6003401F5837426F022900170E0FF74262F5B
:109E0600F582E43401F583E0FFEF9080D493FF9070
:109E16000170E0FE743E2EF582E43401F583EFF026
:099E2600900170E004F0809D221F
:10682E0090023BE0FFEF60030268E490000DE0FF92
:10683E00EF70037F012212A9F5EFB4010312009647
:10684E0012A9F5EF700312005690023AE0FFEFB472
:10685E0001062022037F002290023AE0FFEFB402ED
:10686E0006202F037F002212A9F5EF6401706490B9
:10687E00023AE0FFEF6401702130221EC222E54F82
:10688E00654E600990023B7401F07F00229001106A
:10689E00E0FF90000DEFF07F002290023AE0FFEF54
:1068AE006402702F302F2CC22F90023DE544F090E1
:1068BE00023DE0FF90023CE0FEEE6F600990023B6D
:1068CE007401F07F0022900110E0FF90000DEFF0B8
:1068DE007F00227F002290023BE0FFEF6401600305
:1068EE0002699190000DE0FFEF70037F012212A963
:1068FE00F5EFB4010312009612A9F5EF7003120022
:10690E005690023AE0FFEFB401062022037F0022E8
:10691E0090023AE0FFEFB40206202F037F0022120E
:10692E00A9F5EF6401705A90023AE0FFEFB4011C32
:10693E00302219C222E54FB54E1290023BE4F09080
:10694E000110E0FF90000DEFF07F002290023AE080
:10695E00FFEF6402702B302F28C22F90023DE544CA
:10696E00F090023DE0FF90023CE0FEEEB507129083
:10697E00023BE4F0900110E0FF90000DEFF07F007D
:04698E00227F002242
:10B29E008F7A9000F5E0FF8F36AF7AEF3395E0FEB0
:10B2AE00EF25E0FFEE33FE74542FF58274813EF5E8
:0FB2BE0083E493F508740193F509D229D20C2289
:109EFE007BFF7A8079A112ABFB12539A400B7BFF4A
:109F0E007A8079B212A62180097BFF7A8079C312FA
:109F1E00A6217F17127D70AF321254339000CBE022
:109F2E00FF127D3E9000CCE0FF127D3E9000CDE012
:109F3E00FF127D3E7F1C127D70AF311254339000A4
:109F4E00CBE0FF127D3E9000CCE0FF127D3E9000F4
:079F5E00CDE0FF127D3E2261
:0BB81A007508027509ABD229D20C2280
:0BB8250075081A7509ABD229D20C225D
:10B3E100900107E0FFEF6013900108E0FFE531D322
:10B3F1009F40047F0122227F002222900108E0FF6A
:0DB40100E531C39F50047F0122227F00220D
:10B2CD008F7B9000F7E0FF8F36AF7BEF3395E0FE7D
:10B2DD00EF25E0FFEE33FE74542FF58274813EF5B9
:0FB2ED0083E493F508740193F509D229D20C225A
:05001600C229C20C220A
:0C0096009000FEE0FF8F34D208C2092267
:05005600D208D20922CE
:10B7A500900102E0FFEF600412953B22126992229C
:10953B00900245E0FFEF701612539A4072900105AE
:10954B00E0FF90000FEFF0900245E004F022900254
:10955B0045E0FFEF6401702812539A401C90000FF6
:10956B00E0FFEF704AD25C90010FE0FF90000CEF30
:10957B00F0900245E004F02222900245E4F0222212
:10958B00900245E0FFEFB4022112539A400B900179
:10959B000FE0FF90000CEFF02290000CE0FFEF705B
:1095AB000EC25C900245E4F02222900245E4F022C8
:10699200900245E0FFEF704C900103E0FFEF6023AF
:1069A200900104E0FFE532D39F4013900105E0FF20
:1069B20090000FEFF0900245E004F0228026C25CC6
:1069C200228021900104E0FFE532C39F5013900121
:1069D20005E0FF90000FEFF09002457403F0228073
:1069E20003C25C22900245E0FFEF64017035900122
:1069F20004E0FFEF24FBFFE532D39F401F90000F1E
:106A0200E0FFEF6003026AF5D25C900106E0FF90BE
:106A12000010EFF0900245E004F02222900245E4DB
:106A2200F02222900245E0FFEF6402702E900104F2
:106A3200E0FFEF24FBFFE532D39F400B900106E01D
:106A4200FF900010EFF022900010E0FFEF600302D1
:106A52006AF5C25C900245E4F02222900245E0FF12
:106A6200EF64037043900104E0FF7E00EF2405FF12
:106A7200EE3400FEAD327C00C3ED9FEE6480F8EC94
:106A8200648098501C90000FE0FFEF7066D25C901B
:106A92000106E0FF900010EFF0900245E004F022C2
:106AA20022900245E4F02222900245E0FFEF6404C6
:106AB200703C900104E0FF7E00EF2405FFEE3400FD
:106AC200FEAD327C00C3ED9FEE6480F8EC648098EA
:106AD200500B900106E0FF900010EFF022900010A2
:106AE200E0FFEF700EC25C900245E4F022229002B9
:046AF20045E4F02265
:101F0400202020464C4558204949492020202020A3
:101F14000020202020202020202020202049444C64
:101F240045004E4F204C54522042555320204944E2
:101F34004C45002054657374696E67204D6F646569
:101F44002020200043726F73732042757379204DF3
:101F54006F6465310043726F737320427573792027
:101F64004D6F6465320043726F73732042757379E9
:101F7400204D6F6465330043726F73732042757331
:101F840079204D6F6465340050726F6772616D6DB6
:101F9400696E6757726F6E6700435443535320361C
:101FA400332E302020202020204354435353203606
:101FB400372E3020202020202043544353532036F2
:101FC400392E3420202020202043544353532037DB
:101FD400312E3920202020202043544353532037CE
:101FE400342E3420202020202043544353532037C0
:101FF400372E3020202020202043544353532037B1
:10200400392E372020202020204354435353203896
:10201400322E35202020202020435443535320388F
:10202400352E34202020202020435443535320387D
:10203400382E352020202020204354435353203968
:10204400312E35202020202020435443535320395F
:10205400342E382020202020204354435353203949
:10206400372E342020202020204354435353203142
:1020740030302E302020202020435443535320312D
:1020840030332E3520202020204354435353203115
:1020940030372E3220202020204354435353203104
:1020A40031302E39202020202043544353532031F3
:1020B40031342E38202020202043544353532031E0
:1020C40031382E38202020202043544353532031CC
:1020D40032332E30202020202043544353532031C8
:1020E40032372E33202020202043544353532031B1
:1020F40033312E38202020202043544353532031A1
:1021040033362E352020202020435443535320318E
:1021140034312E3320202020204354435353203184
:1021240034362E3220202020204354435353203170
:1021340035312E3420202020204354435353203162
:1021440035362E372020202020435443535320314A
:1021540035392E3820202020204354435353203136
:1021640036322E3220202020204354435353203132
:1021740036352E352020202020435443535320311C
:1021840036372E3920202020204354435353203106
:1021940037312E3320202020204354435353203101
:1021A40037332E38202020202043544353532031EA
:1021B40037372E33202020202043544353532031DB
:1021C40037392E39202020202043544353532031C3
:1021D40038332E35202020202043544353532031BC
:1021E40038362E32202020202043544353532031AC
:1021F40038392E3920202020204354435353203192
:1022040039322E3820202020204354435353203188
:1022140039362E3620202020204354435353203176
:1022240039392E3520202020204354435353203263
:1022340030332E3520202020204354435353203262
:1022440030362E352020202020435443535320324F
:1022540031302E3720202020204354435353203242
:1022640031382E3120202020204354435353203230
:1022740032352E372020202020435443535320321C
:1022840032392E312020202020435443535320320E
:1022940033332E36202020202043544353532032FE
:1022A40034312E38202020202043544353532032ED
:1022B40035302E33202020202043544353532032E2
:1022C40035342E31202020202020202020202020C2
:1022D400202020202020202020444353203030364A
:1022E40020494E5620303231204443532030303779
:1022F40020494E5620323134204443532030313566
:1023040020494E5620313431204443532030313754
:1023140020494E562030353020444353203032314A
:1023240020494E5620303036204443532030323337
:1023340020494E5620303437204443532030323520
:1023440020494E5620323434204443532030323610
:1023540020494E5620343634204443532030333100
:1023640020494E56203632372044435320303332EE
:1023740020494E56203035312044435320303336E3
:1023840020494E56203137322044435320303433D1
:1023940020494E56203434352044435320303437BA
:1023A40020494E56203032332044435320303530B8
:1023B40020494E56203031372044435320303531A4
:1023C40020494E5620303332204443532030353395
:1023D40020494E562034353220444353203035347E
:1023E40020494E562034313320444353203036356F
:1023F40020494E5620323731204443532030373160
:1024040020494E562033303620444353203037324F
:1024140020494E562032343520444353203037333C
:1024240020494E562035303620444353203037342B
:1024340020494E562031373420444353203131341F
:1024440020494E5620373132204443532031313510
:1024540020494E5620313532204443532031313601
:1024640020494E56203735342044435320313232EC
:1024740020494E56203232352044435320313235E0
:1024840020494E56203336352044435320313331CE
:1024940020494E56203336342044435320313332BE
:1024A40020494E56203534362044435320313334AA
:1024B40020494E56203232332044435320313431A4
:1024C40020494E5620303135204443532031343393
:1024D40020494E5620343132204443532031343580
:1024E40020494E562032373420444353203135326C
:1024F40020494E562031313520444353203135355F
:1025040020494E5620373331204443532031353649
:1025140020494E562032363520444353203136323A
:1025240020494E562035303320444353203136352C
:1025340020494E562032353120444353203137321E
:1025440020494E562030333620444353203137340B
:1025540020494E56203037342044435320323035FE
:1025640020494E56203236332044435320323132F0
:1025740020494E56203335362044435320323134DB
:1025840020494E56203030372044435320323233D2
:1025940020494E56203133342044435320323235BF
:1025A40020494E56203132322044435320323236B1
:1025B40020494E56203431312044435320323433A1
:1025C40020494E562033353120444353203234348D
:1025D40020494E562030323520444353203234357E
:1025E40020494E562030373220444353203234366B
:1025F40020494E562035323320444353203235315E
:1026040020494E562031363520444353203235324A
:1026140020494E5620343632204443532032353537
:1026240020494E5620343436204443532032363128
:1026340020494E5620373332204443532032363318
:1026440020494E562032303520444353203236350B
:1026540020494E56203135362044435320323636F5
:1026640020494E56203435342044435320323731E8
:1026740020494E56203036352044435320323734D7
:1026840020494E56203134352044435320333036CC
:1026940020494E56203037312044435320333131C2
:1026A40020494E56203636342044435320333135A6
:1026B40020494E562034323320444353203332359C
:1026C40020494E562035323620444353203333318B
:1026D40020494E5620343635204443532033333278
:1026E40020494E5620343535204443532033343367
:1026F40020494E5620353332204443532033343658
:1027040020494E562036313220444353203335314C
:1027140020494E5620323433204443532033353637
:1027240020494E562032313220444353203336342C
:1027340020494E562031333120444353203336351B
:1027440020494E562031323520444353203337310B
:1027540020494E56203733342044435320343131FA
:1027640020494E56203232362044435320343132ED
:1027740020494E56203134332044435320343133DE
:1027840020494E56203035342044435320343233CC
:1027940020494E56203331352044435320343331BD
:1027A40020494E56203732332044435320343332A9
:1027B40020494E5620353136204443532034343595
:1027C40020494E5620303433204443532034343689
:1027D40020494E5620323535204443532034353277
:1027E40020494E5620303533204443532034353469
:1027F40020494E5620323636204443532034353552
:1028040020494E5620333332204443532034363249
:1028140020494E5620323532204443532034363436
:1028240020494E5620303236204443532034363526
:1028340020494E5620333331204443532034363616
:1028440020494E5620363632204443532035303307
:1028540020494E56203136322044435320353036F9
:1028640020494E56203037332044435320353136E7
:1028740020494E56203433322044435320353233DA
:1028840020494E56203234362044435320353236C4
:1028940020494E56203332352044435320353332B9
:1028A40020494E56203334332044435320353436A4
:1028B40020494E5620313332204443532035363597
:1028C40020494E5620373033204443532036303687
:1028D40020494E562036333120444353203631327A
:1028E40020494E5620333436204443532036323464
:1028F40020494E5620363332204443532036323753
:1029040020494E562030333120444353203633314E
:1029140020494E5620363036204443532036333235
:1029240020494E5620363234204443532036353421
:1029340020494E5620373433204443532036363210
:1029440020494E56203436362044435320363634FC
:1029540020494E56203331312044435320373033FD
:1029640020494E56203536352044435320373132E2
:1029740020494E56203131342044435320373233DA
:1029840020494E56203433312044435320373331C9
:1029940020494E56203135352044435320373332B5
:1029A40020494E56203236312044435320373334A5
:1029B40020494E5620333731204443532037343393
:1029C40020494E562036353420444353203735347D
:1029D40020494E5620313136204284A4830124C339
:1029E400040274A344C282E364D4430381231463C2
:0F29F40094B4C47D3D1D0D0585C5E5F5FD009529
:10792D00900132E0FFB4010A9000A974FFF0E40267
:10793D0079FAEF640260030279FF12536C7880E6E6
:10794D0060030279EE3054030279EE900238E07054
:10795D0032D22D900119E024FF92499000A8E0FF4A
:10796D009001F9F0900117E09001FAF09001FBEF12
:10797D00F01258B89001FCEFF0128D5D9002387442
:10798D0002F0221284DDEF64017050D22D9001F6C9
:10799D00E0FF24E0F582E43401F583E09001F9F095
:1079AD0074CB2FF582E43401F583E09001FAF09069
:1079BD0001F6E09001FBF01257029001FCEFF09000
:1079CD0001F9E0245BF582E43401F583E024FF92B4
:1079DD0049128D5D900238E014F022900238E014C7
:1079ED00F09000A8E09000A9F0900117E09000AA97
:1079FD00F02290022DE0B40B005046907A0FF8283B
:107A0D002873027A30027A33027A36027A39027A90
:107A1D003C027A3F027A4E027A42027A45027A4855
:107A2D00027A4B022A030271C20273180241BA0292
:107A3D00997E02322302B7C402B7D302B7E202B76E
:077A4D00F1E490022DF0228C
:102A03009000A8E0D39414400302322290022EE0F7
:102A1300B40C00400302321D902A22F828287302C6
:102A23002A46022A5E022C9E022CE5022D02022D6A
:102A330033022E09022E91022F24022F6302302D1E
:102A430002311C7BFF7A1F790412ABFB7BFF7A1FD9
:102A5300791512A62190022E022C9A20552390025A
:102A63006AE0701D204F127BFF7A1F790412ABFBC3
:102A73007BFF7A1F792612A62190026A7402F0C2A4
:102A83004F20A55C12536C900133E060031253781E
:102A9300900130E0900000F09000A8E0FF9000A9C2
:102AA300F0900117E0FE9000AAF090022E7405F05A
:102AB3009001F9EFF09001FAEEF09000A8E0900198
:102AC300FBF01257029001FCEFF0900119E024FF94
:102AD3009249128D5DD22D7BFF7A1F793702ABFBB2
:102AE30012A9F5EF6401705C304659C2469000A408
:102AF300E0FFC39415504D745B2FF582E43401F568
:102B030083E0FFA244E4336F703A12706BA24492E5
:102B1300459000A4E0900232F09000A5E0900233CB
:102B2300F09000A3E0900234F0641F60179002322B
:102B3300E0FF900233E0FD7C00128C1A90022D74AA
:102B43000202314AC24612B57DBF011712536C907F
:102B53000133E06003125378900130E0900000F0FD
:102B6300022F0E900134E0601C12A9F5EF6401609E
:102B73000612B3E1BF010E900111E078A4F69002B2
:102B83002E7409F02212A9F5EF640170683022282F
:102B9300C22290023A04F0D220854E4FE54F75F0E1
:102BA30010A4249DF9741F35F0FA7BFF12ABFBAF21
:102BB3004F129203C220802A302F3AC22F90023C38
:102BC300E544F075F010A424DDF9742235F0FA7BA6
:102BD300FF12ABFB90023CE0FF12905090023A745C
:102BE30002F090022D7405F0E490022EF090011192
:102BF300E078A4F622C222C22F78A6E618467033E4
:102C0300900118E0FF602C75F00AA4A6F008F69076
:102C130000A974FFF09000AAF012536C900133E006
:102C23006003125378900130E0900000F090022E80
:102C33000231AC900123E0FF7003023222900011B5
:102C4300E06003023222900121E0FE601070030273
:102C53003222900240E064016003023222900011AC
:102C6300EFF0E4900240F012536C900133E0600304
:102C7300125378900130E0900000F09000A8E090AB
:102C830000A9F09000AA74FDF0E490022EF09001E8
:102C930022E090022D60647401F022900000E06055
:102CA300030232223054030232229000A8E0FF9044
:102CB30001F9F09001FA74FFF09001FBEFF090013D
:102CC300FCF0900119E024FF9249128D5DD22D2072
:102CD300360920370620380312710D90022E740333
:102CE300F0227880E660030232223054030232225B
:102CF30090010CE0900001F090022E7404F02290F9
:102D03000001E06003023222125372900133E0604B
:102D13000312537EE490022EF090024004F020361A
:102D23000C203709203806127D8D127D9F022DFE5F
:102D330030A503022DF99000A8E09000A9F09001BE
:102D430017E09000AAF012A9F5BF010512009680C2
:102D5300031200567880E6600302322230540302E5
:102D63003222900238E07034D22D900119E024FF12
:102D730092499000A8E0FF9001F9F0900117E090CC
:102D830001FAF09001FBEFF01258B89001FCEFF05C
:102D9300128D5D9002387402F002710D1284DDEF22
:102DA3006401704FD22D9001F6E0FF24E0F582E438
:102DB3003401F583E09001F9F074CB2FF582E4340C
:102DC30001F583E09001FAF09001F6E09001FBF049
:102DD3001257029001FCEFF09001F9E0245BF582B9
:102DE300E43401F583E024FF9249128D5D12710DE5
:102DF300023201023201E490022EF09000A974FF26
:102E0300F09000AAF022900000E06003023222302A
:102E130054030232227880E660030232229000A932
:102E230074FFF09000AAF0128675EF64016003024C
:102E33002F159001F6E0FF24E0F582E43401F583D9
:102E4300E09001F9F074CB2FF582E43401F583E0CF
:102E53009001FAF09001F6E09001FBF012B71790A1
:102E630001FCEFF09001F9E0245BF582E43401F515
:102E730083E024FF9249128D5DD22D20360920373D
:102E83000620380312710D90022E7407F02212A946
:102E9300F5EF6401705F30465EC2469000A4E0FF28
:102EA300C394155052745B2FF582E43401F583E02B
:102EB300FFA244E4336F703F12706BA244924590BB
:102EC30000A4E0900232F09000A5E0900233F0906D
:102ED30000A3E0900234F0641F601C900232E0FF14
:102EE300900233E0FD7C00128C1AE490022EF090E5
:102EF300022D0231ACC2467880E6600302322230F2
:102F0300540302322212B57DEF600790022E74063D
:102F1300F02290010CE0900001F090022E7408F072
:102F230022900001E06003023222125372900133B7
:102F3300E0600312537E9002407401F0E490022E8D
:102F4300F09000A974FFF09000AAF030360302322B
:102F530022303703023222303803023222027D9FAD
:102F630012A9F5EF64017063304660C2469000A475
:102F7300E0FFC394155054745B2FF582E43401F5DC
:102F830083E0FFA244E4336F7041A2449245900072
:102F9300A4E0900232F09000A5E0900233F090009C
:102FA300A3E0900234F012706B900234E0641F606F
:102FB3001A900232E0FF900233E0FD7C00128C1A7B
:102FC300E490022EF090022D0231ACC24678A4E6C2
:102FD30060030232229000A8E09000A9F09000AABA
:102FE30074FDF0900134E0FF64016004EFB4021556
:102FF30012A9F5BF010F900112E090000AF09002B0
:103003002E740AF022900134E0FF64036004EFB4ED
:10301300041512B3E1BF010F900112E090000AF012
:1030230090022E740BF02202321D12A9F5BF010883
:10303300900112E090000AF090000AE0701D125314
:1030430072900118E075F00AA478A5A6F008F6902E
:1030530000A974FFF09000AA02314A900134E0B451
:1030630001097BFF7A1F794802315B12536C7BFFA6
:103073007A1F795912A6217880E6600302320E3056
:10308300540302320E900238E07031D22D900119B0
:10309300E024FF92499000A8E0FF9001F9F090012D
:1030A30017E09001FAF09001FBEFF01258B890018D
:1030B300FCEFF0128D5D9002380231AC1284DDEF2B
:1030C3006401704CD22D9001F6E0FF24E0F582E418
:1030D3003401F583E09001F9F074CB2FF582E434E9
:1030E30001F583E09001FAF09001F6E09001FBF026
:1030F3001257029001FCEFF09001F9E0245BF58296
:10310300E43401F583E024FF9249128D5D0232011C
:10311300900238E014F002320E12B3E1BF010890BE
:103123000112E090000AF090000AE0701E12537240
:10313300900118E075F00AA478A5A6F008F69000AF
:10314300A974FFF09000AAF002321D900134E0B49C
:1031530003097BFF7A1F796A02A6217BFF7A1F7915
:103163007B12A62112536C7880E6600302320E3084
:10317300540302320E900238E07032D22D900119BE
:10318300E024FF92499000A8E0FF9001F9F090013C
:1031930017E09001FAF09001FBEFF01258B890019C
:1031A300FCEFF0128D5D9002387402F0221284DD80
:1031B300EF64017050D22D9001F6E0FF24E0F58218
:1031C300E43401F583E09001F9F074CB2FF582E448
:1031D3003401F583E09001FAF09001F6E09001FBF1
:1031E300F01257029001FCEFF09001F9E0245BF537
:1031F30082E43401F583E024FF9249128D5D90024D
:1032030038E014F022900238E014F09000A8E09027
:1032130000A9F09000AA74FDF022E490022EF0229F
:1071C20090022EE0FF700F900000E0600302731740
:1071D20090022F027311EF6401705F12A3079002F5
:1071E2002FE0D39409400990010CE0900001802027
:1071F20090022FE0FF04F0743E2FF582E43401F593
:1072020083E0900231F0E0FFB4260D900001743269
:10721200F090022E7406F022EFB4240A900124E0CA
:1072220075F0060272C7900231E09029DD93900258
:1072320031F05407900230F0807D90022EE064021B
:10724200703912A307900124E0FF900002F090022F
:1072520031E0FE30E709EF75F003A4900002F0EE92
:1072620025E0900231F0900230E014F0900125E028
:10727200FF12B2CD90022E7403F02290022EE0B4DF
:10728200031E12A307900002E0600302731790012D
:1072920024E0900002F012001690022E7404F022F4
:1072A20090022EE06404702912A307900002E0709D
:1072B20064900230E0600790022E7402F022900186
:1072C20024E075F003A4900002F090022E7405F001
:1072D2002290022EE0B4050B12A307900002E07088
:1072E20034802D90022EE06406702A900001E07036
:1072F20024125372900133E0600312537E900118FE
:10730200E075F00AA478A5A6F008F6E490022DF044
:0673120090022E04F0229F
:1073180090022EE0704F9000E5E0604212536C90AE
:107328000133E06003125378900130E0900000F0E0
:107338009000E6E060229000E9E0B4300F9000E8A9
:10734800E0B430089000E7E064306012206A0FD2A1
:107358006A90022D7407F02290022D0273EA9002BF
:107368002E7404F02290022EE0640170487880E6C2
:10737800600302745E30540302745E900232E0903F
:1073880001F9F0900233E09001FAF09001FB741FCC
:10739800F01257029001FCEFF0A2459249128D5D60
:1073A800D22D20360920370620380312710D90029D
:1073B8002E7402F02290022EE0640270297880E692
:1073C800600302745E30540302745E90010CE09016
:1073D8000001F0203609203706203803127D9F90DF
:1073E800022E7403F02290022EE06403703790009E
:1073F80001E07062125372900133E0600312537E11
:10740800900118E075F00AA478A5A6F008F6E490B3
:10741800022DF07BFF7A1F790412ABFB7BFF7A1FEA
:10742800791502A62190022EE0D394034028E49017
:10743800022DF090022E04F07BFF7A1F790412AB24
:10744800FB7BFF7A1F791512A62112537290013324
:07745800E0600312537E22E5
:1041BA0090022EE0FF7017900232E09000A9F09072
:1041CA000233E09000AAF090022E7401F022EF640C
:1041DA0001705A900000E06003024591A24592499D
:1041EA00900232E09001F9F0900233E09001FAF087
:1041FA009000A8E09001FBF01258B89001FCEFF093
:10420A00128D5DD22D20360920370620380312710F
:10421A000D90010BE090000BF090010DE090001260
:10422A00F09002387408F090022E0242E090022EBA
:10423A00E06402702F126C58EF600280467880E6C4
:10424A0060030245913054030245917628D2549076
:10425A000238E014F0E060030245917402F0900223
:10426A002E04F02290022EE06403600302434A12F5
:10427A006C58EF6002800C90010DE0600D90001206
:10428A00E0700790022E7404F0227880E660030240
:10429A004591305403024591900238E0703CA245A2
:1042AA009249900232E09001F9F0900233E09001D5
:1042BA00FAF09000A8E09001FBF01258B89001FCC7
:1042CA00EFF0128D5DD22D203609203706203803F3
:1042DA0012710D9002387402F0221284DDEF64012B
:1042EA0070579001F6E0FF24E0F582E43401F5838B
:1042FA00E09001F9F074CB2FF582E43401F583E004
:10430A009001FAF09001F6E09001FBF0125702904A
:10431A0001FCEFF09001F9E0245BF582E43401F549
:10432A0083E024FF9249128D5DD22D20360B20376F
:10433A000820380512710D8000900238E014F0222E
:10434A0090022EE0640470342036092037062038A3
:10435A0003127D8D120056E4900239F09000E4E0D9
:10436A006014900131E0FF12B29E78A3761478A30C
:10437A00E670FB12B85A90022E7405F090022EE0F5
:10438A00640570457880E6704020543DA245924904
:10439A00900232E09001F9F0900233E09001FAF0D5
:1043AA009001FB741FF012B7179001FCEFF0128D09
:1043BA005D9002387403F02036092037062038034E
:1043CA0012710D90022E7406F090022EE0FF640620
:1043DA0070297880E67024205421900238E0700F0A
:1043EA0090010CE0900001F090022E7407F0227800
:1043FA00807628D254900238E014F0EF6407600304
:10440A00024591900134E0601F302209302F0612D4
:10441A00B3E1EF7013E490022DF090022EF09001B8
:10442A0011E078A4F602458312A9F5EF640160034E
:10443A000244C22046030244C2C24612A9F5EF64EE
:10444A000170759000A4E0FFC39415506B745B2F44
:10445A00F582E43401F583E0FFA244E4336F705837
:10446A00A24492459000A4E0900232F09000A5E0A8
:10447A00900233F09000A3E0900234F0641F603899
:10448A00900232E0FFC39415502E745B2FF582E43C
:10449A003401F583E0FFA245E433B5071B900232ED
:1044AA00E0FF900233E0FD7C00128C1A90022D741A
:1044BA0002F0E490022EF0227880E67069205466B9
:1044CA00128675EF6401705E9001F6E0FF24E0F554
:1044DA0082E43401F583E09001F9F074CB2FF58280
:1044EA00E43401F583E09001FAF09001F6E09001DE
:1044FA00FBF01257029001FCEFF09001F9E0245B07
:10450A00F582E43401F583E024FF9249128D5D902F
:10451A00022E7406F0E490022DF0203609203706A8
:10452A0020380312710D900001E0705B12537290F3
:10453A000133E0600312537E203609203706203803
:10454A0003127D9F9000A974FFF09000AAF09002D8
:10455A00407401F0E490022DF090022E04F020360F
:10456A00182037152038127BFF7A1F790412ABFB0B
:10457A007BFF7A1F791512A621900118E075F00ABF
:08458A00A478A5A6F008F622B2
:10997E0090022EE0FF7017900000E07067F559F529
:10998E005A9000F8E0F53490022E7401F022EFB4F4
:10999E00011D12A307D20B125DAD5013E4F559C28F
:1099AE000B90010CE0900001F090022E7402F090EA
:1099BE00022EE06402702D12A307900001E07024C5
:1099CE00125372900133E0600312537E900118E03F
:1099DE0075F00AA478A5A6F008F6E490022DF09092
:0599EE00022E04F0222E
:1032230090022EE0600302333912A9F5EF640170B6
:1032330057304654C2469000A4E0FFC3941550484B
:10324300745B2FF582E43401F583E0FFA244E43399
:103253006F703512706BA24492459000A4E0900207
:1032630032F09000A5E0900233F09000A3E09002CA
:1032730034F0641F6012900232E0FF900233E0FDED
:103283007C00128C1A023542C24678A4E66003021F
:10329300387D12A9F5EF640160030233259000D94C
:1032A300E07025125372900133E0600312537E9055
:1032B3000134E0B401109000A8E09000A9F0900060
:1032C300AA74FEF08070806612536C900133E06044
:1032D30003125378900130E0900000F09000A8E0D2
:1032E3009000A9F09000AA74FEF09000DBE0601A51
:1032F300206A09D26A90022D7409F0221253729047
:103303000133E0600312537E802490010DE09000AE
:1033130012F0900110E090000DF090022E7401F075
:103323008014125372900133E0600312537EC22063
:10333300E490022DF02290022EE064016003023338
:10334300D4900000E060030233D490023AE06401B9
:103353007036AF4F12963620367120376E20386B99
:10336300E54F75F010A4249DF9741F35F0FA7BFF27
:1033730012ABFBE54F75F010A4249DF9741F35F0D3
:10338300FA7BFF12A621804390023AE06402704167
:1033930090023CE0FF12188720363020372D20386A
:1033A3002A90023CE075F010A424DDF9742235F074
:1033B300FA7BFF12ABFB90023CE075F010A424DD16
:1033C300F9742235F0FA7BFF12A62190022E0238FF
:1033D3007790022EE06402704112682EEF6014129F
:1033E3007D8D90022E7403F09000D7E070030238B5
:1033F3007D801E90010DE06021900012E0701B1291
:103403007D8D90022E7403F09000D7E07003023894
:103413007D90011DE0900004F02290022EE06403F1
:10342300600302354A900004E07048127D9F120049
:1034330056E490023BF09000D7E06014900131E035
:10344300FF12B29E78A3761978A3E670FB12B85ADE
:103453009000D8E0600F90011EE090000EF0900203
:103463002E7404F02290011FE0900003F012B800C4
:1034730002356612A9F5EF6401705A12B8003022C2
:103483002CC22290023A7401F0C220854E4F20369E
:1034930019203716203813E54F75F010A4249DF931
:1034A300741F35F0FA7BFF12ABFB02359A302F25E0
:1034B300C22F90023CE544F0203617203714203801
:1034C3001175F010A424DDF9742235F0FA7BFF1294
:1034D300ABFB0235C6C222C22F12A9F5EF640170FD
:1034E3006430466112B800C220C2469000A4E0FFD7
:1034F300C394155050745B2FF582E43401F583E0D7
:10350300FFA244E4336F703D12706BA24492459066
:1035130000A4E0900232F09000A5E0900233F09016
:1035230000A3E0900234F0641F601A900232E0FFBF
:10353300900233E0FD7C00128C1AE490022EF0908E
:10354300022D023877C24690022EE0640460030223
:10355300364E90000EE0701112B80090011FE090FB
:103563000003F090022E0237FD12A9F5EF640170FB
:103573006B12B800302230C22290023A7401F085F7
:103583004E4FC220E54F75F010A4249DF9741F35EA
:10359300F0FA7BFF12ABFBAF4F129203E490022EC3
:1035A300F090022D0237FD302F32C22F90023CE5FE
:1035B30044F075F010A424DDF9742235F0FA7BFF92
:1035C30012ABFB90023CE0FF12905090023A74025F
:1035D300F0E490022EF090022D0237FDC222C22F9A
:1035E30012A9F5EF6401706130465E12B800C22083
:1035F300C2469000A4E0FFC39415504D745B2FF5B1
:1036030082E43401F583E0FFA244E4336F703A129D
:10361300706BA24492459000A4E0900232F09000B7
:10362300A5E0900233F09000A3E0900234F0641F11
:103633006017900232E0FF900233E0FD7C00128CB1
:103643001A90022D74020236CBC24690022EE06419
:10365300056003023744900003E0700790022E7464
:1036630006F02212A9F5EF6401706430222BC22206
:1036730090023A04F0854E4FC220E54F75F010A436
:10368300249DF9741F35F0FA7BFF12ABFBAF4F1289
:10369300920390022D7405802F302F33C22F900296
:1036A3003CE544F075F010A424DDF9742235F0FAFA
:1036B3007BFF12ABFB90023CE0FF12905090023A6A
:1036C3007402F090022D7405F0E490022EF022C2F1
:1036D30022C22F12A9F5EF6401706430466112B85B
:1036E30000C220C2469000A4E0FFC394155050745A
:1036F3005B2FF582E43401F583E0FFA244E4336FEA
:10370300703D12706BA24492459000A4E090023287
:10371300F09000A5E0900233F09000A3E090023413
:10372300F0641F601A900232E0FF900233E0FD7CE8
:1037330000128C1AE490022EF090022D023877C208
:103743004690022EE06406600302387D900001E09B
:10375300703F125372900133E0600312537E7BFF7C
:103763007A1F790412ABFB7BFF7A1F791512A6210E
:10377300900118E075F00AA478A5A6F008F6900267
:10378300407401F0C220E490022DF090022E04F068
:103793002212A9F5EF6401706530222CC222900237
:1037A3003A04F0854E4FE54F75F010A4249DF9744B
:1037B3001F35F0FA7BFF12ABFBAF4F129203E4907D
:1037C300022EF090022D8032302F33C22F90023C14
:1037D300E544F075F010A424DDF9742235F0FA7B8A
:1037E300FF12ABFB90023CE0FF12905090023A7440
:1037F30002F0E490022EF090022D7405F022C22212
:10380300C22F12A9F5EF6401706E30466B12B80037
:10381300C220C2469000A4E0FFC39415505A745BC3
:103823002FF582E43401F583E0FFA244E4336F70A3
:103833004720360920370620380312706BA24492C2
:10384300459000A4E0900232F09000A5E09002338E
:10385300F09000A3E0900234F0641F601B900232EA
:10386300E0FF900233E0FD7C00128C1AE490022EFC
:0B387300F090022D7402F022C24622E9
:0FB7C4007BFF7A1F798C12ABFBE490022DF022F1
:0FB7D3007BFF7A1F798C12ABFBE490022DF022E2
:0FB7E2007BFF7A1F798C12ABFBE490022DF022D3
:0FB7F1007BFF7A1F798C12ABFBE490022DF022C4
:1045920043544353532036332E30202020202020F2
:1045A20043544353532036372E30202020202020DE
:1045B20043544353532036392E34202020202020C8
:1045C20043544353532037312E39202020202020BA
:1045D20043544353532037342E34202020202020AC
:1045E20043544353532037372E302020202020209D
:1045F20043544353532037392E3720202020202084
:1046020043544353532038322E352020202020207B
:1046120043544353532038352E3420202020202069
:1046220043544353532038382E3520202020202055
:1046320043544353532039312E352020202020204B
:1046420043544353532039342E3820202020202035
:1046520043544353532039372E3420202020202026
:104662004354435353203130302E30202020202019
:104672004354435353203130332E35202020202001
:104682004354435353203130372E322020202020F0
:104692004354435353203131302E392020202020DF
:1046A2004354435353203131342E382020202020CC
:1046B2004354435353203131382E382020202020B8
:1046C2004354435353203132332E302020202020B4
:1046D2004354435353203132372E3320202020209D
:1046E2004354435353203133312E3820202020208D
:1046F2004354435353203133362E3520202020207B
:104702004354435353203134312E33202020202070
:104712004354435353203134362E3220202020205C
:104722004354435353203135312E3420202020204E
:104732004354435353203135362E37202020202036
:104742004354435353203135392E38202020202022
:104752004354435353203136322E3220202020201E
:104762004354435353203136352E35202020202008
:104772004354435353203136372E392020202020F2
:104782004354435353203137312E332020202020ED
:104792004354435353203137332E382020202020D6
:1047A2004354435353203137372E332020202020C7
:1047B2004354435353203137392E392020202020AF
:1047C2004354435353203138332E352020202020A8
:1047D2004354435353203138362E32202020202098
:1047E2004354435353203138392E3920202020207E
:1047F2004354435353203139322E38202020202075
:104802004354435353203139362E36202020202062
:104812004354435353203139392E35202020202050
:104822004354435353203230332E3520202020204E
:104832004354435353203230362E3520202020203B
:104842004354435353203231302E3720202020202E
:104852004354435353203231382E3120202020201C
:104862004354435353203232352E37202020202008
:104872004354435353203232392E312020202020FA
:104882004354435353203233332E362020202020EA
:104892004354435353203234312E382020202020D9
:1048A2004354435353203235302E332020202020CE
:1048B2004354435353203235342E312020202020BC
:1048C20020202020202020202020202020202020E6
:1048D20044313233343536373839302A2341424372
:107B780075840F12554A12B4BA9000A8E0FF600548
:107B8800D3941440069000A87401F0128AC912A177
:107B98004012A19C12B3B4125394129FC81253728C
:107BA800123D31900118E0FF78A5760008A607E499
:107BB80090018BF090022EF090022DF0900239F097
:107BC80090023EF0129DC6E4900241F0900011F040
:107BD800125384D2ACD2A830311D12B53012B4BAC7
:107BE800128AC912A14012A19C12B3B4C236C2377C
:107BF800C23812387E80E0120056127D9F20A32CD6
:107C0800303F12C23F787EE6540F9048D2939001DD
:107C18008AF01295BB3040E5C240787CE6540F905C
:107C280048D293900189F01296B180D120A4051210
:107C38009EFE80F81288B6304126C24112B5301235
:107C4800B4BA128AC912A14012A19C12B3B4C236A6
:107C5800C237C238129FC8E490022DF090022EF06D
:107C6800203606203703303805127DB180F243E70D
:107C780040900013E0700E305508129F6512B557FA
:107C880080031290E312792D1249C61276D812B7E2
:037C9800A580992B
:105A58008DB7948A98419BDC9F3AA27EA5A9A8BAE3
:105A6800ABB1AEA5B150B40DB614B800BA6FBCD680
:105A7800BF14C148C365C577C74FC95FCB41CD0BBC
:105A8800CEC1D072D20DD2F2D39CD47FD51ED5F818
:105A9800D693D764D7FAD8C3D955DA16DAA8DB6112
:105AA800DBE9DC9FDD22DDD4DEFDE019E093E12EA9
:105AB800E239E33CE3AA0000000000000000000017
:105AC80000000000000000000000000000000000CE
:105AD80000000000000000000000000000000000BE
:105AE80000000000000000010000000000010000AC
:105AF800000000010000000000000001000000009C
:105B0800000100000000000100000000000100008A
:105B1800000000010000000000010000000000017A
:105B2800000000000001000000000001000000016A
:105B38000001000000010001000000010001000058
:105B48000001000100000000000100010000000148
:105B58000001000000010001000000010001000038
:105B68000001000100000001000100000001000127
:105B78000000000100010000000100010000000118
:105B88000001000000010001000000010001000008
:105B980000010001000000010001000000010001F7
:105BA80000000001000100000001000100000001E8
:105BB80000010000000100010000000100010000D8
:105BC80000010001000000010001000100010001C6
:105BD80000010001000100010001000100010001B5
:0E5BE8000001000100010001000100010001A8
:10963600C22BC22DD2B3D2B275F006EFA424BEF56A
:1096460082E5F0345AF583E493FC740193FDEC4D06
:1096560024FF92B075F006EFA424C0F582E5F0343D
:109666005AF583E493FC740193FDEC4D24FF92B705
:1096760075F006EFA424C2F582E5F0345AF583E4CA
:1096860093FC740193FDEC4D24FF92B5EF25E02485
:1096960058F582E4345AF583E493F52E740193F574
:0B96A6002FD22CE4F584D28CD2A92234
:0EB80000C22BC22DC22CE4F584C28CC2A92238
:104F160020504C55472050484F4E454C494E452051
:104F260000554E504C55472050484F4E454C494E23
:104F36004500504C5547494E2050484F4E454C4928
:104F46004E450044313233343536373839302A232A
:104F560041424302AB055508000AAB0D551000123D
:104F6600AB155518001AAB1D55200022AB25552848
:104F7600002AAB2D55300032AA3555202054455312
:104F86005420524F5554494E452020202056455214
:104F960053494F4E20312E30202020205445535463
:104FA600494E4720454550524F4D202020544553E9
:104FB60054494E4720564F494345202054455354A3
:104FC600494E472044544D462031202054455354E1
:104FD600494E472044544D46203220202054455304
:104FE60054494E47205253323332202020544553E1
:104FF60054494E47205253343835202020205445FA
:105006005354494E4720505454202020544553545D
:10501600204155582052454C41592020544553545F
:105026002043542052454C41592020205445534991
:105036004E472052494E47494E47202020202020E7
:10504600202020202020202020202020544553549A
:10505600204C494E45204C4F4F5020544553542028
:105066004C494E452053454E53452B5445535420E9
:105076004C494E452053454E53452D5445535420D7
:105086004C494E4520494E205553452054455354CE
:1050960020494E50555420564F4C54205445535495
:1050A600204C494E452052454C41595445535420B5
:1050B6005A45524F2043524F535320544553544957
:1050C6004E4720535155454C4348202020544553C4
:1050D60054494E47204850462020202054455354DA
:1050E6002054454C434F20564F5820205445535486
:1050F60020524144494F20564F582020202020203E
:105106002020202020202020202020202020202099
:105116002020202020202020202020202020202089
:1051260020202020202020202020202054455354B9
:1051360020434F4D504C4554454420202020544593
:0B5146005354204641494C45442020B2
:10387E007BFF7A4F798112ABFB7BFF7A4F799112E6
:10388E00A62112B8467BFF7A4F79A112ABFB127DAF
:10389E009F12B846E4FFFE1275E0900170EFF07DC6
:1038AE00AAE4FFFE12759FE4FFFE1275E0EF64AA14
:1038BE00600C7BFF7A51794112A6211200717D5561
:1038CE00E4FFFE12759FE4FFFE1275E0EF64556093
:1038DE000C7BFF7A51794112A62112007190017072
:1038EE00E0FDE4FFFE12759F7BFF7A51793112AB3A
:1038FE00FB12B8467BFF7A4F79B112ABFB12538C99
:10390E0012B830E4F559755A01789E7614125DA4FA
:10391E00789EE670FB125D9B12B85AE4F559755A03
:10392E0001789E7605789EE670FBD202D20B125D70
:10393E0092C202C20B7BFF7A51793112ABFB12B8E5
:10394E00467BFF7A4F79C112ABFB127D9F12B846B0
:10395E00C2277F3112B6AD789E761E789EE670FB3A
:10396E0012B8613027FD787EE6547F904F49937BE5
:10397E00FFB4310C7A51793112ABFB12B846800A82
:10398E007A51794112A6211200717BFF7A4F79D1BB
:10399E0012ABFB127D9F12B8467F3112B69612B84B
:1039AE005012B8613025FD787CE6547F904F4993D4
:1039BE007BFFB4310C7A51793112ABFB12B84680D1
:1039CE000A7A51794112A6211200717BFF7A4F7942
:1039DE00E112ABFB127D9F12B846E4F58475985048
:1039EE00C299C2987599433098FDE4F584E59964BF
:1039FE0043600C7BFF7A51794112A6211200717B34
:103A0E00FF7A51793112ABFB12B8467BFF7A4F79B0
:103A1E00F112ABFB127D9F12B846125397E4F58458
:103A2E00759850C299C2987599433099FD7BFF7A6B
:103A3E0051793112ABFB12B8467BFF7A50790112E5
:103A4E00ABFB127D9F12B84612536C12B850E53282
:103A5E00D39432400C7BFF7A51794112A621120089
:103A6E007112537212B850E532C394AA500C7BFFF8
:103A7E007A51794112A6211200717BFF7A51793168
:103A8E0012ABFB12B8467BFF7A50791112ABFB12C8
:103A9E007D9F12B84612537812B850E531D3940A6E
:103AAE00400C7BFF7A51794112A6211200711253FC
:103ABE007E12B850E531C394AA500C7BFF7A51792F
:103ACE004112A6211200717BFF7A51793112ABFBA4
:103ADE0012B8467BFF7A50793112ABFB127D9F12E2
:103AEE00B8461253AF40FB7BFF7A51793112ABFBD4
:103AFE0012B8467BFF7A50795112ABFB127D9F12A2
:103B0E00B84612538412B8501253BB501A1253C1F6
:103B1E0040157BFF7A50796112ABFB1253BB40FB11
:103B2E001253C150F6801D1253BB50DC1253C140CC
:103B3E00D77BFF7A50797112ABFB1253BB40FB124D
:103B4E0053C150F67BFF7A51793112ABFB12B84656
:103B5E0012538C7BFF7A50798112ABFB127D9F1230
:103B6E00B84612538C1253B550107BFF7A4F79160C
:103B7E0012A6211253B540FB800E7BFF7A4F792798
:103B8E0012A6211253B550FB127D9F7BFF7A5179FD
:103B9E003112ABFB12B84612538C7BFF7A507991DF
:103BAE0012ABFB127D9F12B846E530C3940A400754
:103BBE00E530D3943C400C7BFF7A51794112A6211B
:103BCE001200717BFF7A51793112ABFB12B8467B32
:103BDE00FF7A5079A112ABFB127D9F12B846125399
:103BEE008412B8501253A6400B7BFF7A4F793812CD
:103BFE00ABFB80F07BFF7A51793112ABFB12B846EA
:103C0E0012538C7BFF7A5079B112ABFB127D9F124F
:103C1E00B84612B81A1253AC40FB1253AC50FB12FA
:103C2E0053AC40FB7BFF7A51793112ABFB12B84695
:103C3E0012B85A7BFF7A5079C112ABFB127D9F12DC
:103C4E00B84612539A400B12536C12537212539A77
:103C5E0050F57BFF7A51793112ABFB12B8467BFFE0
:103C6E007A5079F112ABFB127D9F12B84612B8252D
:103C7E001253A050FB12B85A7BFF7A51793112AB16
:103C8E00FB12B8467BFF7A5079D112ABFB127D9FA7
:103C9E0012B84612B81A12B748904F5B12B73F903F
:103CAE004F5D12B73F904F5F12B73F904F6112B703
:103CBE003F904F6312B73F904F6512B73F904F67DB
:103CCE0012B73F904F6912B73F904F6B12B73F90AC
:103CDE004F6D12B73F904F6F12B73F904F7112B7A3
:103CEE003F904F7312B73F904F7512B73F904F777B
:103CFE0012B73F904F7912B73F904F7B12B73F905C
:103D0E004F7D12B73F904F7FE493F508740193F502
:103D1E000912B85A7BFF7A51793112ABFB12B846B1
:033D2E00023CA1B3
:0AB84600789E760A789EE670FB22D9
:0AB85000789E7602789EE670FB22D7
:09B73F00E493F508740193F50987
:0AB74800789E7605789EE670FB22DD
:0200710080FE0F
:0300A30002A9B2FD
:10A9B200C0E0C0F0C083C082C0D075D000C000C06B
:10A9C20001C002C003C004C005C006C0072055056F
:10A9D200128337800312A50BD007D006D005D0040E
:10A9E200D003D002D001D000D0D0D082D083D0F01A
:03A9F200D0E03280
:03009300029C8844
:099C8800C0E0C0D075D000C00797
:109C9100AF84758402E543700885BE3375BB0780C8
:109CA10032E543B4010885BE3075BB048025E54328
:109CB100B4020885BE3375BB068018E543B40308BA
:109CC10085BE3175BB04800BE543B4040A85BE3300
:109CD10075BB0505438010E543B4050885BE3275A3
:0B9CE100BB048000754300C2ED8F84BF
:079CEC00D007D0D0D0E03218
:0300830002AC3399
:10AC3300C0E0C0F0C083C082C0D075D000C000C0E7
:10AC430001C002C003C004C005C006C007C2CF12C2
:10AC53001700D007D006D005D004D003D002D0010E
:0DAC6300D000D0D0D082D083D0F0D0E0322D
:03007B0002A08759
:10A08700C0E0C0F0C083C082C0D075D000C000C09F
:10A0970001C002C003C004C005C006C00720240FCA
:10A0A70085BF4085BE3FD22475BB01C2ED801385B5
:10A0B700BF3E85BE3DC22430580312817E75BB006A
:10A0C700C2EDD007D006D005D004D003D002D0010E
:0DA0D700D000D0D0D082D083D0F0D0E032C5
:03007300028FBC3D
:108FBC00C0E0C0F0C083C082C0D075D000C000C07B
:108FCC0001C002C003C004C005C006C007C2CF78F0
:108FDC009AE6600116302E27124C29C22ED55C055C
:108FEC00755C0A055BD51B09751B0A7584014388E2
:108FFC0020D51C19751C60758402438820800ED204
:10900C002E789B16E670067604F584D28B305505C7
:10901C00129E2F800312A3B612929012981C758484
:10902C0001438810758400D2ECD007D006D005D04F
:10903C0004D003D002D001D000D0D0D082D083D0C5
:04904C00F0D0E0324E
:03006B000287F613
:1087F600C0E0C0F0C083C082C0D075D000C000C049
:0D88060001C002C003C004C005C006C007C9
:1088130085841620261875840F30DF3875840FE59C
:10882300E8540F787CF6D226787D76C88026787D4A
:1088330016E6700E75840FE5E8540F787CF6E6446F
:1088430080F675840F20DF0CC226D225D240D26277
:10885300D25FD26820281630F833E5E854F0FFC41D
:10886300540F787EF6D228787F76C88020787F16DA
:10887300E6700FE5E854F0FFC4540F787EF6E64443
:1088830080F620F808C228D227D23FD26112745F43
:08889300758402C28D85168474
:10889B00D007D006D005D004D003D002D001D00031
:0B88AB00D0D0D082D083D0F0D0E032DB
:03005B0002A1F807
:10A1F800C0E0C0F0C083C082C0D075D000C000C02D
:10A2080001C002C003C004C005C006C0071248FB55
:10A21800789CE6600116E5416002154190000CE06B
:10A22800600214F0900247E0600214F0758401C2E5
:10A238008DD007D006D005D004D003D002D001D0ED
:0CA2480000D0D0D082D083D0F0D0E03223
:0300530002A85FA1
:10A85F00C0E0C0F0C083C082C0D075D000C000C0BF
:10A86F0001C002C003C004C005C006C007C28C30BF
:10A87F005A04C25A8005D25A124D48D007D006D07A
:10A88F0005D004D003D002D001D000D0D0D082D0D8
:06A89F0083D0F0D0E0328E
:03002B0002000FC1
:03000F00C2CF322B
:03001B0002006E72
:03006E00C28F320C
:0300130002AE1129
:10AE1100C0E0C0F0C083C082C0D075D000C000C007
:10AE210001C002C003C004C005C006C0071213E878
:10AE3100D007D006D005D004D003D002D001D00075
:0BAE4100D0D0D082D083D0F0D0E0321F
:10AAB800191823A01296203D129623A012962763F8
:10AAC8001488203D148823A01488276316B8203DD5
:10AAD80016B823A016B827631918203D191827633C
:10AAE80012962B8C14882B8C16B82B8C19182B8C3F
:0BB8300075081575095ED229D20322AD
:0BB83B0075081575095ED229D20C2299
:07B85A00C229C203C20C2247
:10B69600E4F512F513F514F5159000F3E0F53512FF
:07B6A6006F13D22AD2042227
:10B6AD00E4F512F513F514F5159000F4E0F53512E7
:07B6BD006F13D22AD20D2207
:106F1300EF127F8B700E236FFD2A6F4B306F5D3145
